:020000040800F2
:100000000040002049760008357600083776000861
:1000100000000000000000000000000000000000E0
:100020000000000000000000000000003976000819
:1000300000000000000000003B7600083D7600084C
:100040009976000899760008997600089976000854
:10005000997600089976000899760008955F00085F
:100060009976000899760008997600089976000834
:100070009976000899760008D52F0008997600082F
:100080009976000899760008997600089976000814
:100090009976000899760008997600089976000804
:1000A0009976000899760008997600083D4A00087C
:1000B000812A000899760008997600089976000848
:1000C00010B5064C2378002B07D1054B002B02D02E
:1000D000044800E000BF0123237010BD2800002069
:1000E00000000000C48F0008044B10B5002B03D0A3
:1000F0000349044800E000BF10BDC04600000000F6
:100100002C000020C48F00080023C25C0133002AA9
:10011000FBD1581E7047000002B4714649084900DF
:10012000095649008E4402BC7047C04602B471466D
:1001300049084900095C49008E4402BC7047C0462A
:10014000002243088B4274D303098B425FD3030A16
:100150008B4244D3030B8B4228D3030C8B420DD329
:10016000FF22090212BA030C8B4202D312120902B7
:1001700065D0030B8B4219D300E0090AC30B8B42F5
:1001800001D3CB03C01A5241830B8B4201D38B03A3
:10019000C01A5241430B8B4201D34B03C01A524148
:1001A000030B8B4201D30B03C01A5241C30A8B428B
:1001B00001D3CB02C01A5241830A8B4201D38B0276
:1001C000C01A5241430A8B4201D34B02C01A52411A
:1001D000030A8B4201D30B02C01A5241CDD2C3098C
:1001E0008B4201D3CB01C01A524183098B4201D308
:1001F0008B01C01A524143098B4201D34B01C01AF3
:10020000524103098B4201D30B01C01A5241C3086A
:100210008B4201D3CB00C01A524183088B4201D3D9
:100220008B00C01A524143088B4201D34B00C01AC5
:100230005241411A00D20146524110467047FFE731
:1002400001B5002000F0F0F802BDC0460029F7D04B
:1002500076E7704703460B437FD4002243088B4266
:1002600074D303098B425FD3030A8B4244D3030B3D
:100270008B4228D3030C8B420DD3FF22090212BA02
:10028000030C8B4202D31212090265D0030B8B427E
:1002900019D300E0090AC30B8B4201D3CB03C01A68
:1002A0005241830B8B4201D38B03C01A5241430B43
:1002B0008B4201D34B03C01A5241030B8B4201D333
:1002C0000B03C01A5241C30A8B4201D3CB02C01A9E
:1002D0005241830A8B4201D38B02C01A5241430A16
:1002E0008B4201D34B02C01A5241030A8B4201D305
:1002F0000B02C01A5241CDD2C3098B4201D3CB01AC
:10030000C01A524183098B4201D38B01C01A52415A
:1003100043098B4201D34B01C01A524103098B425E
:1003200001D30B01C01A5241C3088B4201D3CB0049
:10033000C01A524183088B4201D38B00C01A52412C
:1003400043088B4201D34B00C01A5241411A00D2DC
:1003500001465241104670475DE0CA0F00D0494245
:10036000031000D34042534000229C4603098B42B5
:100370002DD3030A8B4212D3FC22890112BA030A3D
:100380008B420CD3890192118B4208D389019211BF
:100390008B4204D389013AD0921100E08909C30944
:1003A0008B4201D3CB01C01A524183098B4201D346
:1003B0008B01C01A524143098B4201D34B01C01A31
:1003C000524103098B4201D30B01C01A5241C308A9
:1003D0008B4201D3CB00C01A524183088B4201D318
:1003E0008B00C01A5241D9D243088B4201D34B0033
:1003F000C01A5241411A00D20146634652415B1075
:10040000104601D34042002B00D549427047634655
:100410005B1000D3404201B5002000F005F802BD9A
:100420000029F8D016E770477047C046D0400B004F
:10043000D1409C46203AD3401843524263469340F1
:1004400018437047844608006146FFE71FB500F077
:100450009FFB002801D40021C8421FBD10B500F049
:100460002BFB4042013010BD10B500F091FB00287D
:1004700001DB002010BD012010BDC04610B500F00A
:1004800087FB002801DD002010BD012010BDC04603
:1004900010B500F037FB002801DC002010BD012062
:1004A00010BDC04610B500F02DFB002801DA002079
:1004B00010BD012010BDC046F0B5CE469946030CD4
:1004C0009C46130447461B0C1D000E0061460404A5
:1004D000240C80B50700100C4B4365434143604337
:1004E0002C0CC01820188C46834203D980235B0251
:1004F0009846C444494679435643030C2D042D0CB9
:100500008919634400044019C918C0BCB946B046F3
:10051000F0BDC0469E2110B5C905041CFFF7C2FFFF
:10052000002803D1201C00F065FE10BD9E21201C78
:10053000C90500F0BFFC00F05DFE80231B069C4651
:100540006044F2E7F8B54746CE464A02430245000A
:10055000C40F500A804648005B0A000E9209944678
:1005600080B51E00814602002D0EDF00C90F8C42AF
:1005700024D0281A00280EDD002A3ED16246002A27
:1005800000D1FDE0421E012800D137E1FF2800D153
:10059000A9E0100039E0002863D04B46521B002D23
:1005A00000D0E0E0002F00D1CEE0531E012A00D1A0
:1005B00055E1FF2A00D194E01A00D9E02A1A002A56
:1005C00000DC99E0002862D0FF2D00D18BE0802371
:1005D0006146DB0419438C461B2A00DCD2E0012370
:1005E000DB195A016AD50135FF2D5BD00122A349E1
:1005F0001A405B080B4013431CE0FF2D00D172E052
:1006000080236246DB041A4394461B2800DC90E0FA
:100610000123FB1A5A0151D59B019E09300000F0BD
:10062000A3FE330005388340854200DC75E0944A20
:100630002D1A13405A0704D00F221A40042A00D062
:1006400004335A013CD5681CFE2D2BD09B015E0A59
:10065000C0B2C0053043E4072043C0BCB946B04631
:10066000F8BDFE206A1C104272D1002D00D0AEE011
:10067000002F00D1ECE063460020002BE9D0FB1AEC
:100680005A0100D4F3E063460C00DB1BD2E761465D
:1006900000295BD0511E012A00D1A7E0FF2A22D0F9
:1006A0000A0099E7FF200026D3E7FE216A1C1142C9
:1006B00073D0FF2AF6D0150067447B085A07BBD1D8
:1006C000DB08FF2D0FD05B025E0AE8B2C1E762468D
:1006D000002A08D08022D203134204D040461042A0
:1006E00001D10C004346002BDCD08026F6031E43CC
:1006F0007602FF20760AACE7002AD6D0421B002DF6
:100700005CD0FF28EED08023DB041F431B2A00DCD3
:1007100082E001234D46634463E72022401B013001
:10072000121A19009340C1405A1E934100250B43F1
:1007300080E7202361461B1A994062460B00C240A5
:10074000591E8B41134364E70C0043461500B8E77C
:100750006346FE1A730145D4002E00D05EE70024E4
:100760000020002675E7FF2BBBD08023DB041F434E
:100770001B2A47DD012362460C004D46D31A49E788
:1007800005009EE761462023D1409B1A62469A40AD
:1007900013005A1E93410B4322E7002D46D1002F30
:1007A00062D063460020002B00D152E73B00634437
:1007B0005A0183D5324A013513407FE7002FC4D058
:1007C000531E012A12D0FF2A8CD01A009EE7002F58
:1007D00000D07CE76346002B83D180260024FF20D5
:1007E000F60336E763460C00DE1B17E73B00634465
:1007F00001255A0100D461E70225F7E66346012589
:10080000FB1A07E720239B1A38009F403B00D0408B
:100810005A1E93410343AEE720239B1A39009F40A1
:100820003B00D1405A1E93410B4373E7002F00D188
:1008300058E76246002A00D155E78022D2031342CE
:1008400000D150E74146114200D04CE743464AE709
:100850006346002B83D00C0046460020F9E6634631
:100860000C00DB1B0135D5E646460020F1E6002BE7
:1008700000D023E700240026EBE6C046FFFFFF7D03
:10088000FFFFFFFBF0B54F464646D6464502C0B5D2
:1008900047000C1C6D0A3F0EC60F002F00D16FE001
:1008A000FF2F00D174E00023802299469A46ED0084
:1008B000D20415437F3F63025B0A984663001B0E18
:1008C000E40F002B4DD0FF2B45D042468021D200B3
:1008D000C9041143884600227F3B3100FF1A4B4672
:1008E0006140C9B20F2B00D9B8E070489B00C358D3
:1008F0009F46002398462600454692465346022BC3
:1009000000D18DE0032B00D1A1E0012B18D03B00DA
:100910007F33002B6DDD6A0704D00F222A40042AA2
:1009200000D004352A0103D5614B1D403B008033C4
:10093000FE2B00DD74E0AA01520AD8B202E00E00DC
:1009400000200022C005F60710433043E0BCBA4641
:10095000B146A846F0BD4346002B3FD10222FF3FDF
:1009600003E04346002B2DD1012231004B4661406C
:10097000C9B213430F2B38D84E489B00C3589F462B
:10098000002D13D104239946033B00279A4692E792
:10099000002D05D108239946063BFF279A468AE792
:1009A0000C239946093BFF279A4684E7280000F06C
:1009B000DBFC7627431F9D4000237F4299469A46E1
:1009C0003F1A78E7404600F0CFFC4246431F9A406A
:1009D00076235B4290461B1A00227EE703234A4699
:1009E0001A439146FC33032277E70E00FF200022D2
:1009F000A8E70122D31A1B2BA2DC9E372A00BD4098
:100A0000DA406B1E9D4115436A0704D00F222A402D
:100A1000042A00D004356A0144D50120002291E760
:100A2000FF2000228EE780220026FF20D20389E7E4
:100A3000002398468022D203154208D04346134231
:100A400005D11A4352022600FF20520A7AE780227B
:100A5000D2032A435202FF20520A73E742466B0137
:100A60005501AB421AD21B200022013F01261C0077
:100A700052005B00002C01DB9D4201D85B1B32431E
:100A800001380028F3D1581E834113431D003B0059
:100A90007F330E00002B00DD3DE7AAE71A2001227C
:100AA0005B1BE3E7AA010020520A4BE7DC8F00083A
:100AB000FFFFFFF71C90000870B5420045024E0290
:100AC0004C00C30F6D0A0120120E760A240EC90FC6
:100AD000FF2A06D0FF2C03D0A24201D1B54206D096
:100AE00070BD002DFCD1FF2CFAD1002EF8D18B4225
:100AF00006D00120002AF3D12800431E9841EFE7D9
:100B00000020EDE770B5420045024E024C00C30FD5
:100B10006D0A120E760A240EC80FFF2A1BD0FF2C76
:100B20000ED0002A1BD1002C01D1002E1CD0002D8C
:100B30000CD083421CD00221581E0840013870BDE1
:100B4000002E22D1002AF4D1002DF2D10028F6D1B6
:100B500001204042F3E7002D17D1FF2CF0D0002CEC
:100B6000E7D1002EE5D1E6E70020002DE7D0E2E74F
:100B7000A24205DCEADBB54202D8E7D30020DEE77B
:100B80004342584140000138D9E702204042D6E7AD
:100B900070B5420045024E024C00C30F6D0A120EA2
:100BA000760A240EC80FFF2A0BD0FF2C0DD0002A86
:100BB0001FD1002C16D1002E14D10020002D10D0F2
:100BC00009E0002D0CD1FF2C13D1002E08D1002AF2
:100BD00008D0834212D00221581E0840013800E09C
:100BE000022070BD002DF4D10028FAD1012040422E
:100BF000F7E7002CEDD1002EEBD1ECE7A24205DCAB
:100C0000F2DBB54202D8EFD30020EAE74342584175
:100C100040000138E5E7C04643025B0AF0B54F46A5
:100C200046469946D646C30F45009846C0B54B4642
:100C30000F1C2D0E00D1CBE0FF2D00D1CFE0802284
:100C4000DB00D2041A430023914600269A467F3DDA
:100C50007C027B00640A1B0EFF0F002B00D1A9E071
:100C6000FF2B11D08022E400D204144342467F3B84
:100C70005B197A400020D2B25D1C0A2E13DD3A00C7
:100C80000B2E47D047463FE02B00FF33002C1ED1F0
:100C900002221643424601357A40D2B2FF350A2E6F
:100CA00000DDE4E00220022E1CDC013E012E42D8D1
:100CB00002283DD0012866D100200021C00508434C
:100CC000D2071043E0BCBA46B146A846F0BD0322A5
:100CD0001643424601357A40D2B2FF350A2E00DD76
:100CE000E4E003200121B140A626F60031420AD1FA
:100CF0009026B600314216D1B93EFF3E0E421AD0C0
:100D0000A146824600E0170053463A00022B0FD05E
:100D10004C4650460328CDD18021C90321434902C6
:100D2000FF20490ACAE780210022FF20C903C5E746
:100D3000FF200021C2E7200C49462404240C270090
:100D40000E0C0904090C74434F4346434843390CC5
:100D5000001909188C4203D9802040028446664459
:100D60003F0408043F0CC0198401671EBC41090CF4
:100D7000800E8919044389010C43090171D50123AF
:100D800061081C400C432B007F33002B51DD6107B1
:100D900004D00F212140042900D00434210103D5BF
:100DA000434B1C402B008033FE2BC1DCA101490AC0
:100DB000D8B283E7002C2CD1012342461E432B00DE
:100DC0007A400120D2B25D1C0A2E00DD57E76AE7A7
:100DD000002B10D10123042600259A4638E7002B6A
:100DE00004D102230826FF259A4631E703230C2667
:100DF000FF259A462CE7484600F0B6FA4A46431FBC
:100E000076259A4000236D42914600269A462D1A77
:100E10001EE7200000F0A8FA4246431F9C402B1A10
:100E2000763B7A400020D2B25D1C0A2E00DD26E718
:100E300039E70121CB1A1B2B00DD3DE79E35210050
:100E4000AC40D940631E9C4121434B0704D00F2383
:100E50000B40042B00D004314B0104D501200021AC
:100E60002CE71D008FE789010020490A26E70223AD
:100E70000F2E0CD180214B46C9030B420DD00C42E2
:100E80000BD1214349023A00FF20490A16E70B2EF5
:100E900000D0F7E6A1469A4636E780214B46C903C3
:100EA000194349024246FF20490A07E70323DFE7C7
:100EB000FFFFFFF7F0B5C64643025B0A4500DA00C4
:100EC000C40F48024F009446420A1E00904600B5E7
:100ED0002D0E3F0EC90F8009FF2F59D0012251401E
:100EE0008C4239D0EA1B002A58DD002F68D0FF2D34
:100EF00000D1D1E08023DB0418431B2A00DCE3E0AF
:100F000001236246D31A5A0100D4ACE09B019E092A
:100F1000300000F029FA330005388340854200DCB8
:100F2000C6E0B24A2D1A13405A0704D00F221A40C5
:100F3000042A00D004335A0100D497E06A1CFE2D25
:100F400000D184E09B015E0AD2B2D0053043E407B1
:100F5000204380BCB846F0BDEA1B002A41DD002FCB
:100F60006BD0FF2D00D197E08023DB0418431B2AB0
:100F700000DCCCE0012363445A0174D50135FF2D18
:100F800065D001229A491A405B080B401343CBE716
:100F900000281FD08C4222D02A00FF3A002A35D0E8
:100FA0007A1B002D00D099E06346002B00D1DDE0D4
:100FB000531E012A00D105E1FF2A6BD01A0094E0EC
:100FC000002873D0511E012A00D1DFE0FF2A63D030
:100FD0000A0092E701225140A14200D082E72A0094
:100FE000FF3A002A36D07A1B002D00D1AAE0FF2F4D
:100FF00000D1DAE080236146DB0419438C461B2ACA
:1010000000DCD4E001233D001B18B5E7FE276A1C75
:10101000174271D1002D00D09EE06346002B00D115
:10102000D5E00022002800D18FE71B1A5E0100D412
:10103000D6E063460C00C31A76E7002836D0511E6E
:10104000012A00D19AE0FF2A26D00A008FE7FF226A
:1010500000267AE7FE276A1C174262D0FF2AF6D0E4
:101060001500604443085A0700D05FE7DB08FF2DF6
:1010700012D05B025E0AEAB267E76246002A00D13C
:1010800093E0002808D08022D203134204D04046C7
:10109000104201D10C004346002BD8D08026F60325
:1010A0001E437602FF22760A4FE743461500DEE72D
:1010B0002022401B0130121A19009340C1405A1ED1
:1010C000934100250B432FE720239B1A01009840F2
:1010D0000300D1405A1E93410B4312E7FF2FD9D092
:1010E00080236446DB041C43A4461B2A52DD0123F3
:1010F0000C003D00C31A06E763461E1A730139D47B
:10110000002E00D004E70024002200261DE7202343
:101110009B1A010098400300D1405A1E93410B4393
:1011200029E7002DA9D16346002B56D000220028C4
:1011300000D10AE7030063445A0194D52B4A0135D4
:10114000134090E76346002BAFD0531E012A15D001
:10115000FF2A2AD01A0052E76246002A91D10028BD
:1011600098D180260024FF22F603EEE60C004346C9
:1011700015007CE763460C00C61AC9E60300634409
:1011800001255A0100D46EE70225FAE663460125DF
:101190001B1AB8E664462023D4409B1A62469A4044
:1011A00013005A1E93412343A2E7434674E7614666
:1011B0002023D1409B1A62469A4013005A1E934145
:1011C0000B4320E763460C000125C31A9BE6002869
:1011D00099D00C0046460022B7E646460022B4E607
:1011E000002B00D03FE700240026AEE6FFFFFFFB08
:1011F000FFFFFF7D41024200C30F490A0020120E8B
:101200007E2A03DD9D2A02DD094A98187047802056
:1012100000040143952A07DC9620821AD1404842F7
:10122000002BF3D10800F1E7963A9140F7E7C0466A
:10123000FFFFFF7F70B5002813D0C317C5185D40AE
:10124000C40F280000F090F89E2301001B1A962B73
:101250000FDC082831D008398D406D026D0AD8B2F4
:1012600002E0002400200025C0052843E4072043B5
:1012700070BD992B0CDD0522121A2800D040020007
:1012800008001B3085402800451EA8410243150078
:10129000052916DC2A000F4802406E0709D00F26E8
:1012A0003540042D05D00432550102D59F2302405C
:1012B0005B1A9201550AD8B2D6E76D0296206D0AE4
:1012C000D2E74A1F95402A00024802406E07F0D03C
:1012D000E5E7C046FFFFFFFB70B5041E0ED000F02F
:1012E00043F89E2301001B1A962B0CDC08282CD0F7
:1012F00008398C406402640AD8B201E0002000245E
:10130000C005204370BD992B0ADD020020001B326E
:1013100090400200501E82410520401AC4401443F0
:10132000052916DC22000F480240650709D00F2569
:101330002C40042C05D00432540102D59F230240D6
:101340005B1A9201540AD8B2DAE764029620640A62
:10135000D6E74A1F94402200024802406507F0D0B9
:10136000E5E7C046FFFFFFFB1C2101231B04984259
:1013700001D3000C10391B0A984201D3000A083926
:101380001B09984201D30009043902A2105C4018DD
:101390007047C04604030202010101010000000081
:1013A000000000004B425941002343708370013319
:1013B000C370013303710133017043717047437887
:1013C0008B420DD0417001290BD0022914D0002985
:1013D0001DD10123C370DB18037181700133437188
:1013E00070470378002B0AD001238370DB18C37089
:1013F000002303710333F2E70378002BF4D00223B8
:1014000083700023C370013303710233E7E7FEE703
:1014100013B56A460B8813804B8853808B88938062
:10142000CB88D380831C06306C461A780133520077
:10143000A25A0A8002318342F6D113BD4018807847
:101440007047000003000B4AA03370B51A60020019
:10145000012300257F210400A4325B4255711380D3
:101460009170AC30B834D380063200F0FFFC2570A8
:1014700070BDC0467F7F7F7F70B5040011001500EE
:101480001E0000F096FC20002900143000F091FCB2
:1014900020002900283000F08CFC200029003C307E
:1014A00000F087FC20002900503000F082FC200072
:1014B0002900643000F07DFC20002900783000F025
:1014C00078FC200029008C3000F073FCFA23200007
:1014D000190032005B00C900AC3000F0AFFC200006
:1014E000FFF7B0FF70BD704710B500F069FC10BD8C
:1014F00010B5143000F064FC10BD10B5283000F0B9
:101500005FFC10BD0300A4331B78002B03D1A03077
:10151000007840B27047A130FAE70300A4331B788B
:10152000002B03D1A230007840B27047A330FAE715
:1015300010B5040004F060FF0023984208D020009A
:10154000143000F041FC031C002800D10123DBB261
:10155000180010BD10B5040004F04EFF002398429F
:1015600008D02000503000F02FFC031C002800D1D0
:101570000123DBB2180010BDFA2110B5AC30890090
:1015800000F07BFC10BD10B50021AC3000F075FC04
:1015900010BD10B5AC3000F081FCFA239B009842DE
:1015A00001DD180010BDC343DB171840FAE710B582
:1015B000040000F0D9FB2000143000F0D5FB20001F
:1015C000283000F0D1FB20003C3000F0CDFB2000A3
:1015D000503000F0C9FB2000643000F0D3FB200045
:1015E000783000F0CFFB10BD030000207F2B08D027
:1015F0000130002B05DA1A007E30803201D05B42C8
:10160000D8B2704703007F20002B01D05B4258B254
:101610007047030010B5FF207F2B10D01A0001384F
:1016200031320CDA1A000020783208DB78335BB2F2
:10163000FE30584346212330FEF70CFEC0B210BDE9
:101640000300FF207F2B07D00138002904D00020A1
:10165000834201DA5B42D8B270470000030010B544
:1016600000207F2B10D01A0031320EDA1A00AC3075
:10167000783209DB064878335BB258434621233081
:10168000FEF7E8FDAC3080B210BD0248FCE7C04672
:10169000A906000055070000030010B5632808D80C
:1016A0000548642158433230FEF74AFDAC3080B221
:1016B00010BD0248FCE7C046A9060000550700001F
:1016C000064B10B5C318F020C00058430449FEF77C
:1016D000C1FDF8239B00C01880B210BD00FCFFFFC5
:1016E000FF07000010B5FFF7EBFF10BD064B10B56C
:1016F000C3189620C00058430449FEF7ABFD044BC5
:10170000C01880B210BDC04600FCFFFFFF070000FC
:10171000DC050000054B0322C0180F234343D817F4
:101720001040C018801000B27047C04600FCFFFF98
:1017300003000020032B18DD01300C2B15DD0130D8
:101740000F2B12DD0630122B0FDD0538162B0CDDAA
:101750000430192B09DD03381C2B06DD01301F2B4B
:1017600003DDFA30212B00DCF93870470300FF203D
:10177000052B01D8014AD05C7047C046A9900008EB
:10178000030000207F2B01D05B42D8B270470000DD
:1017900010B5002A09D08A18044C92B20B78013196
:1017A00058408BB2205C9A42F8D110BDB09000082E
:1017B0000300392809D80020222B05D90848233BEB
:1017C000DBB2D84001231840704701205F2BFBD0CB
:1017D00000201922613BDBB29A424041C0B2F3E7DC
:1017E00001EC7F00F7B504000F0006000025831D03
:1017F00001933078FF2801D10135EDB2FFF7D8FF12
:10180000002801D15F233370019B0136B342F0D130
:10181000062D06D1002F04D02A003900200007F041
:10182000C7FB0023A371F7BDF0B5831D85B000226F
:101830000393002304000126002500920193114F19
:101840003800217807F068FB002801D0C31BD8B20C
:1018500032002B000021FEF72FFE009A019B121888
:101860004B41300000920193290000232822FEF70B
:1018700023FE039B013406000D00A342E0D1009833
:1018800005B0F0BDB091000810B5417908003038BE
:10189000C3B2092B04D80521FEF7C2FDC8B210BDA2
:1018A000054C200007F038FB002801D0031BD8B2FC
:1018B0000521FEF7CBFCF1E7B091000870B50400FC
:1018C000FEF722FC002382B2501EE118834205DBA2
:1018D000D21A2000013207F0F7FA70BD0D78302DD2
:1018E000F6D101339BB2F0E7F0B50C009BB01500C8
:1018F00000211A001F00060007F0F9FA00212A2231
:1019000003A86D00029107F0F2FA63190193019B9D
:10191000A3420FD102A8FEF7F7FB002804D002ABC8
:10192000C018002301380370300002A907F038FB0B
:101930001BB0F0BD0023E05E234B9842EAD00028A4
:1019400013DC22490EA807F02BFB02A8FEF7DCFBF4
:1019500005000EA8FEF7D8FB2D18AF4203D30EA941
:1019600002A807F0CCFA0234D1E7FA239B00984290
:101970000BDA0EA980B206F091FF0EA8FFF79EFFCA
:1019800013490EA807F0BBFADFE764213230FEF7F7
:1019900061FC0EA980B206F081FF0EA8FFF78EFF52
:1019A0000EA8FEF7B1FB302102AA431E5218D25CEA
:1019B00002AD6D1802392A54E9540EAB18180023F1
:1019C00004494370DDE7C046FF7F00005C900008DB
:1019D0006190000866900008F0B5002489B00231DB
:1019E000E5B2AA4204D86946FFF77EFF09B0F0BD10
:1019F0006F46A6008E5B65007E530134F0E7000061
:101A000070B50B490400FEF721FC20000D000849C9
:101A1000FEF796FB642104032800FEF717FC28005C
:101A200064186421FEF78CFB8001201880B270BD21
:101A30001027000070B50E0000210500140007F00B
:101A400056FA00239AB2944200D870BDF25C002A84
:101A5000FBD0EA540133F5E7030010B508000B4949
:101A6000052805D8FEF762FB03080A0C0E1008498A
:101A70001800FFF7DFFF10BD0649F9E70649F7E751
:101A80000649F5E70649F3E70649F1E788900008BB
:101A90006A9000086F900008749000087990000820
:101AA0007E90000883900008030010B508000B49E1
:101AB000052805D8FEF73AFB03080A0C0E10084962
:101AC0001800FFF7B7FF10BD0649F9E70649F7E729
:101AD0000649F5E70649F3E70649F1E7889000086B
:101AE0008A9000088F900008949000089990000850
:101AF0009E900008A290000870B50E00140000210E
:101B00000132050007F0F3F900239AB2944200D89D
:101B100070BDF25C002AFBD0EA540133F5E7000007
:101B20007D234380044B09B2C36000230180818080
:101B3000C38003727047C046393000000268044B0E
:101B40005343044A9B185B005A080260580C7047C4
:101B5000FD430300C39E2600F0B5002599B0016047
:101B6000858004005622290002A807F0C0F901264A
:101B7000E27DAA4208D8002320008021A375B83056
:101B800007F0B5F919B0F0BD2000FFF7D7FFE779EE
:101B9000791BFEF745FC00221000CBB20193D3B2B3
:101BA0009F4222D8002300221100277BD0B2874217
:101BB00026D80029DCD1A2796119033A012A07D974
:101BC000002D05D017228A56002A20D1012BCFD90B
:101BD0000B76A268990089582A000E3292001151A2
:101BE000013502AAD654EDB2C2E702A9895C0029E8
:101BF00004D101998842D6D00130C0B20132CEE77B
:101C00002069805C984200D131000132CEE7501E3D
:101C10008342DDDB01329342DADCA9E7F0B515003F
:101C200004009DB00160027143715622002106A894
:101C3000013D059307F05BF9EBB2E6790193022BC6
:101C400014D830000321FEF77BFA0323C6B20393B6
:101C500000273D00E27DAA420DD80023200080210C
:101C6000A375B83007F043F91DB0F0BD012303930D
:101C700000230193ECE72000FFF760FF711BFEF7E4
:101C8000CFFB0022CBB202931300D0B2864206D91A
:101C900006A9515C002926D102998B4221D1321C20
:101CA000864200D9021C039BD2B253430199CB1840
:101CB000DBB20293237B9C4600230493D8B2844575
:101CC00013D8049B002BC5D1029BA16805989B00EB
:101CD000C91801380B68032815D8FEF727FA0F2911
:101CE0002B2D0133DBB20132CFE720690299C05CB2
:101CF000884201D1012104910133DFE714481B1808
:101D000014488342A6D9002D03D0002F18D1012AF0
:101D1000A0D90298631918762B0009680E339B002E
:101D20001951012106AB6D1817009954EDB291E7D6
:101D30000948E4E70948E2E709481B180948E0E7D1
:101D40007B1E9A42E5DB7B1C9A42E2DC82E7C046BE
:101D5000C54E47FF3BB10100776245FF287643FF40
:101D60003CB142FF3CB1010070B583684568040096
:101D7000EB1AC3606420618A5843FEF7E1F9A5605D
:101D8000207470BD426883688260D31AC360704754
:101D900010B5416804000020814205D06423E0684A
:101DA0005843FEF7CDF9C0B200232074E3606360AE
:101DB00010BD00234182C360836043600374704799
:101DC0004368013343607047007C704743685B1889
:101DD00043607047002343608360C36003747047AF
:101DE000F8B50D0003601900037C04001600012BF8
:101DF00012D9C76883684268FA20EB1AB21A8000C9
:101E000050431A007A43C918801AFEF723FAC01902
:101E1000E0606660A560F8BD002B03D1C3600133AC
:101E20002374F6E74368FA20A168D31A8000584368
:101E3000691AFEF70FFA0223E060F1E7F7B5050033
:101E4000100014001E000191FFF746FA019B071CC9
:101E5000E018FFF741FA011C381CFEF713FD6E6015
:101E600028603000FFF7E6F9A860F7BD10B5040060
:101E70004068FFF7DFF9A06010BD70B50400A568E9
:101E80000800FFF7D7F9291CFFF714F82168FEF7BF
:101E9000C3FE291CFEF756FBA06070BDFC2110B5E7
:101EA00089058068FEF74EFBFFF7A4F910BD704767
:101EB000704770470020704770470020704700202F
:101EC000704770470020704700207047054B82B074
:101ED0005A6902435A615B6918400190019B02B044
:101EE0007047C04600100240054B82B0DA690243D9
:101EF000DA61DB6918400190019B02B07047C0466F
:101F000000100240054B82B09A6902439A619B69B6
:101F100018400190019B02B07047C046001002407B
:101F2000EFF31082012383F31088802103688B4331
:101F3000036082F310887047044B1888044B1B8899
:101F4000C01A431E984180B27047C046A8140020B2
:101F5000A6140020704700000388044A5940C9B203
:101F600049008A5A1B0A534003807047F4A60008B0
:101F700070B5002A0FD08A180688074D94B20B78E6
:101F8000320A7340DBB25B00EE5A013156408BB22D
:101F90000680A342F3D170BDF4A6000837B5012333
:101FA0006A460C0005005B42D380013C064BA4B29C
:101FB0009C4202D16B46D8883EBD6B462978981D5D
:101FC000FFF7CAFF0135F0E7FFFF000090238022F2
:101FD000DB0512029A62704790238022DB05120211
:101FE0009A61704710B5FFF7A7FF431E9841C0B232
:101FF00010BD00000023044A1380044A1380044AE1
:102000001380044A13807047A6140020A8140020EF
:10201000AA160020AC16002000207047704710B5AB
:10202000FFF78AFF431E9841C0B210BD70B50B4C3C
:102030000622210005000A310948FFF75DFD094B22
:10204000227CFF331209DA76627C1207120F1A77AC
:10205000637ADB0701D502232B7370BD910A002040
:10206000B6010020A4000020064B9A8CEFF31081EB
:10207000012282F3108818681F3202431A6081F32C
:102080001088704700440040FD22F0B5060085B07E
:1020900001AB02701A702732825C04000C36801883
:1020A000012A3DD800255A705D80627065808A7A69
:1020B0001A7122718A7A01328A7262795A71A2790E
:1020C0009A71A2681202120ADA71111212141972AC
:1020D0005A726B460921581DFFF760FF6B46588006
:1020E0006778981CBAB23100FFF742FF2423FF3310
:1020F000E15C6B46981CFFF72FFF6B465A88230064
:10210000FE33DA8192235B00E25C974206D238000C
:102110000C302900D21B201806F0E9FE05B0F0BDF6
:10212000C57A0138002DBDD1013AD2B2B8E700001E
:10213000002310B5064A074C07480849138023803E
:1021400003800B801380238003800B8010BDC0466A
:10215000A6140020A8140020AA160020AC16002007
:1021600013B56B460268D97107331469190001224F
:10217000A04713BD70B5040008000D00FDF7C4FFB3
:102180002368290082B21B692000984770BD0000B7
:10219000902310B5DB050400984209D1802080020D
:1021A000FFF794FE0F4B9C420CD18020C00307E048
:1021B0000D4B984207D00D4B984207D18020000369
:1021C000FFF784FE10BD8020C002E9E7084B98426B
:1021D00002D180204003F3E7064B9842E2D18020F1
:1021E0008003EDE7001400480004004800080048A0
:1021F000000C0048001000481B4B10B5040098422A
:102200000BD180200001FFF77DFE184B9C420ED1C0
:1022100080204002FFF776FE25E08023DB05984210
:102220000BD0134B98420CD10220FFF75DFE114BEF
:102230009C420CD180208002ECE70120FFF754FE85
:10224000E3E70D4B984208D11020FFF74DFE0B4BF2
:102250009C4208D18020C002DCE7094B9842D4D1CF
:102260002020FFF741FE10BD002C0140004001403E
:1022700000040040004401400010004000480140BC
:1022800000140040F0B50E0089B000930EAB1F782B
:102290000FAB1B78050014000021142203A8019342
:1022A00006F025FE02960B2C23D82000FDF73EFFFA
:1022B000060609131515151717171B1D032303937E
:1022C00001E002230693009B032B21D81800FDF7A1
:1022D0002DFF11131D110123F4E70123EFE7012363
:1022E00003930593EFE70223E9E702230393013BFE
:1022F000F7E7FEE703230493082F1BD83800FDF708
:1023000015FF1A1A080D0F11131517000123F2E714
:10231000FEE701230793022303930EE00223F9E76C
:102320000323F7E70423F5E70523F3E70623F1E7A3
:102330000723EFE7FEE7002FEDD1019B002B02D032
:102340002800FFF725FF601F042805D8FDF7EEFEE3
:10235000030A04030A00AE62280002A905F0C4FEC5
:1023600009B0F0BDAE61F7E713B501240194002474
:102370000094FFF787FF13BD70B586B016006B465B
:102380000022DA8004000D00FFF736FF042E37D854
:102390003000FDF7CBFE2529032D36001A4B1B49D3
:1023A0001868FDF7CDFE80B2002301A9013808802E
:1023B0002000CB604B608D600B6106F037F8802207
:1023C0002368134993432360A3680B407021A360E3
:1023D00063688B436360A3689343A36006B070BDDA
:1023E000094B0C491868DCE7074B0B491868D8E71C
:1023F000054B08491868FDF7A3FE0A235843D2E7A6
:10240000FEE70120D0E7C0461C00002080A8120192
:10241000F8BFFFFF40420F0000127A0010B5040021
:10242000FFF7AAFF012322681343236010BD012197
:1024300010B500224942FFF7F1FF10BD174B10B550
:102440001B68174C236005F029F99020C00505F0A2
:10245000E5FD144805F0E2FD134805F0DFFD1348E3
:1024600006F034F9124806F031F905F08FFE00222B
:10247000104B1A605A609A6072B601230E4A5B4292
:10248000D367C0220D4952008B5062B60C4B1B68BB
:1024900083F3088823689847FEE7C04604C8FF1FF7
:1024A000F402002000040048000800480038014001
:1024B0000044004010E000E004E100E000E100E042
:1024C00000C8FF1F70B50849084C081BEFF30883CC
:1024D0005D1E0022A84202D8621AD218013AAA212F
:1024E00006F005FD70BDC04600400020000400005D
:1024F00070B59024E4052000032306220121FFF794
:1025000033FF032380210F4D994028000222FFF75B
:102510002BFF032328001A004021FFF725FF20008E
:10252000032305221021FFF71FFF280003230522A4
:102530000221FFF719FF0323052220212000FFF7C6
:1025400013FF70BD00040048024B18694006C00F1D
:102550007047C0460004004810B5FFF7F5FF00289B
:1025600000D110BDC046F8E70222044B9A629023C6
:102570001E32DB059A61103A9A61704700040048E8
:1025800090231022DB059A6292189A62014B1E3A40
:102590009A617047000400481249134B0A69C12030
:1025A0001A4080235B0013430B61104B10495A689B
:1025B00080000A405A601A680A401A60DA680A40C5
:1025C000DA6080229968D2000A4380219A60094A21
:1025D000090613581B021B0A0B4313508023136078
:1025E0007047C04600000140FFF0FFFF00040140BB
:1025F000FFFBFFFF00E100E08023034ADB005361A3
:1026000011680B4313607047000401400122064B20
:102610000648196891431960596801405960196862
:102620000A431A607047C04600380140FFFFFDFFB3
:1026300001228020054B8002196891431960596876
:102640000143596019680A431A6070470038014015
:10265000902010B5002303228021C005FFF784FEDF
:1026600010BD90230120DB051B69DB0998437047EF
:10267000802110B50A4C0023200006224900FFF7F4
:1026800073FE2000002306228021FFF76DFE8021CB
:102690000023062220008900FFF766FE10BDC04619
:1026A000000400488022054952044869030413408D
:1026B00080225200824313438B617047000400481C
:1026C0008022054912044869030413408022824392
:1026D00013438B617047C0460004004890200023DC
:1026E00003228021C00510B5FFF73EFE9021102285
:1026F00000238020C9050C69044201D10133DBB2FB
:10270000013AD2B2002AF6D10C2B01D9FFF796FE7E
:1027100010BD000010B50248FFF789FE10BDC0468D
:1027200000140040044901304A6A80B292B24B6AF8
:102730009B1A8342FBD37047001400401FB500234F
:10274000029001936946013301A8039305F004F94F
:10275000431E9841043005B000BD0A00002301006B
:1027600010B5022005F090F8431E9841043010BDCA
:1027700010B5FFF7E3FF04384342584180B210BD63
:1027800010B5FFF7EAFF04384342584180B210BD4C
:10279000F0B50E00140085B0012813D03C27254B5E
:1027A000254D0293254B019305F026F839002800AA
:1027B000FFF7DEFF00280CD1002405F031F82000DF
:1027C00005B0F0BD1C4B3D2702931D4B194D0193E5
:1027D000EAE7002E01D1FC24E4000334A410A3B2E4
:1027E0002C00002703931034039ABBB29A4207D8F7
:1027F00028001449FFF7C4FF431E98418400DCE71A
:10280000002E08D1029B5B1B1B1919684B1C05D1BC
:1028100001370434E8E7BB00F158F7E7019B9C421D
:1028200005D22000FFF7ACFF0028F1D1C4E7032454
:10283000C3E7C04600E8010800E00108FFE701081F
:10284000FFEF01081111111110B504F0D5FF3C2163
:102850000848FFF78DFF0024A04206D03D2106481E
:10286000FFF786FF431E9841840004F0D9FF200043
:1028700010BDC04600E0010800E80108002310B5C3
:10288000074C9AB2914201D8042010BDA34205D052
:10289000044A9A181278C2540133F2E70320F4E78D
:1028A000EF07000010E0010870B504000D0072B6DB
:1028B0000A0001000020FFF76BFF62B6042806D172
:1028C00072B62A0021000338FFF762FF62B670BDBE
:1028D000104B70B51D68104B1C68104B9D4208D101
:1028E0000420AC4204D0002211000338FFF750FF4F
:1028F00070BD9C4203D1002211001000F6E7FFF7E3
:10290000A3FF0428F4D12C40013463425C41601CD5
:10291000EEE7C04600E0010800E8010811111111BE
:102920000122044B187399681142FCD0187BC0B285
:102930007047C04600300140F8B506000F00150092
:102940000024AC4200D1F8BD305DFFF7E9FF3855F7
:102950000134F6E710B5080011001A00FFF7ECFF8C
:1029600010BD000070B505000C00002C00D170BD3A
:10297000044B013C1878FFF7D3FFA4B2287001354F
:10298000F3E7C0461400002010B508001100FFF75F
:10299000E9FF10BD70B505000C00002C00D170BD22
:1029A0002878013CFFF7BCFF0135A4B2F5E710B56C
:1029B00008001100FFF7EEFF10BD000030B58DB02C
:1029C0002822002102A806F092FA80258020902477
:1029D0002D02E4054001FFF795FA290020000323AA
:1029E0000622FFF7C1FCA561012403230A22082166
:1029F000204801940094FFF745FC03230A2220217C
:102A00001C4801940094FFF73DFC032310211A0099
:102A1000184801940094FFF735FC8222520003927B
:102A2000FC3200230792E0220825134CD2000593C4
:102A30000693029309930A932000073302A9049294
:102A40000B93089505F0B4FC102263689343636010
:102A50006368AB436360402322681343236002230F
:102A6000A2681A42FCD0FF22237B044B1A700DB0DF
:102A700030BDC04600040048003001401400002072
:102A800020231A4A70B5D069184211D01168194232
:102A90000ED0174C918C174D23882D8801335B0580
:102AA00089B25B0D9D4203D0134DC9B2E954238016
:102AB0001F2313626133184212D0116819420FD0DC
:102AC0000E4B0F4918880B8898420AD00B880133A7
:102AD000DB05DB0D0B800B880A499BB2CB5C1385B1
:102AE00070BD0248FFF71CFAFAE7C04600440040F8
:102AF000A8140020A6140020A60C0020AC1600206C
:102B0000AA160020AA1400200D4902000B880D48C7
:102B100010B501330488DB050020DB0D9C420ED08C
:102B20000948C2540B80EFF31081012080F3108814
:102B30008023064A14682343136081F3108810BD74
:102B4000AC160020AA160020AA1400200044004061
:102B500070B504004518AC4200D170BD2078FFF775
:102B6000D3FF0134F7E710B508001100FFF7F0FFBD
:102B700010BD0000064B074A1B8812889B1A98B2AA
:102B80001B0403D580231B01C01880B27047C046C8
:102B9000A8140020A614002010B5FFF7EBFF10BD0D
:102BA0000848094A018813889942FBD013880133E9
:102BB0005B055B0D13801388044A9BB2D05CC0B2E6
:102BC0007047C046A8140020A6140020A60C0020C0
:102BD00010B5FFF7E5FF10BD70B50C0088B006001A
:102BE00015000021082206A806F081F923005A1ECC
:102BF00093411B0302930C2301A9044801960395FA
:102C00000494059305F0ACFD08B070BD004400408D
:102C100070B50125044C2368AB432360FFF7DCFF4C
:102C200023681D43256070BD00440040002210B59C
:102C300008001100FFF7ECFF10BD000073B501257F
:102C400080203B4C800223680226AB432360FFF7C1
:102C50004BF99020009603230A2204210195C00518
:102C6000FFF710FB032390201A000096082101951E
:102C7000C005FFF707FB0022E12011004002FFF72B
:102C8000ABFF63682B4AC72113402A22FF206360F1
:102C9000A36889009343284AA36053583E36834370
:102CA0003343535080235B0513602000FFF738F94E
:102CB000EFF3108285F310882368B343236082F317
:102CC000108800231D4A266213801D4A1380EFF3EB
:102CD000108185F31088202022688243226081F3CE
:102CE0001088184A80211380174A8903138063686B
:102CF000164A134008226360A3689343A360636885
:102D0000134A134022226360A3689343A360802385
:102D1000A2685B011343A36023681D4380232560E1
:102D2000DB03E2690A42FCD0E2691A42F9D073BDC2
:102D300000440040FFB7FFFF00E100E0AA160020BA
:102D4000AC160020A6140020A8140020FFF7FFFFF7
:102D5000FFBFFFFF10B5FFF771FFFFF785F910BD4B
:102D600010B5FFF7F7FF10BD024B1A68024B1A604F
:102D70007047C046B016002034030020054B064AB9
:102D8000196813680020994202D0013313600130A2
:102D90007047C046B016002034030020034A044B9D
:102DA00011681B785B1813607047C046B01600208E
:102DB0002000002010B50248FFF739FB10BDC046C7
:102DC00000440140014B586A80B270470044014002
:102DD00010B5FFF7EFFFFFF7C7FF10BDF8B507000D
:102DE00015000C003E0004F007FDAD00ED19AE42E9
:102DF00004D1042404F014FD2000F8BDE31B99590C
:102E000033688B4201D10436F1E73000FFF7B8FC9C
:102E10000028F8D10400EDE7037807B5002B0ED0A9
:102E2000074B1A68FA23DB009A4208D300230222D8
:102E300003706946406800930193FFF7CFFF07BD19
:102E4000B0160020012373B50380284B284A196867
:102E50000400914206D1274A5968914202D10023C9
:102E6000037073BD22482349234A18605960002328
:102E70002248234D6360036841685E1C03D093427F
:102E800001D0002B03D14B1C0BD0914209D008304C
:102E9000A842F0D172B63E211848FFF769FC62B62D
:102EA00016486060036842680093591C03D1531CA4
:102EB00019D1114B10E010498B4205D1511C0AD099
:102EC0009A4210D1002307E0002B0CD18A420AD18C
:102ED0008022520022801A00019269460222009349
:102EE000FFF77CFFBDE700232370F4E7000000201C
:102EF00012345678FEDCBA90AAAAAAAA00F00108F9
:102F000000F8010809490B88002B00D1FEE772B6D2
:102F1000074B09885A6A891864325963DA630322B5
:102F200052421A61063A1A6162B6704744000020A4
:102F3000002C0140012110B5134C88B02000032261
:102F40004942FFF76BFA20220021684605F0CFFFC7
:102F500064236A4601212000039305F0B7FA80211B
:102F6000C8236A4620004900039305F0AFFAC32145
:102F7000064B89005A58064802405A508022D20116
:102F80001A6008B010BDC046002C014000E100E00E
:102F9000FFFF00FF0222044BD9680A43DA600822CF
:102FA000D9680A43DA607047002C014064224A4322
:102FB000064B10B51A8004000022054B1A70FFF76B
:102FC000B9FF2000FFF7E6FF10BDC0464400002017
:102FD000310300200C4B1A6992070AD50322524292
:102FE0001A615A6B6432DA63084A596B12885218B4
:102FF0005A631A69120705D5092252421A61044B15
:103000000A321A707047C046002C0140440000206C
:1030100031030020F8B51A4C90220021201D05F044
:1030200066FF072301270025164E63800833310011
:10303000A380052214481D332780FEF7CDFC134BD7
:1030400031006363023B0522A36311482C23A5874B
:10305000FEF7C2FC0F4B1049E366230070331F805C
:1030600023000E4872331D706567A56705F098FF51
:1030700023007F2291331A70052392342370F8BD08
:1030800060020020C89300086602002002000100D0
:103090009E020020020007004E920008DC02002081
:1030A00070B5084C4518415C200005F035FF031E43
:1030B00005D0001B0130C3B2272B00D90023E35CED
:1030C0002B7070BDDC93000870B50D00110004007A
:1030D000160005F065FF002D13D0681E082808D8DB
:1030E000FDF724F80510121416181A1C1E003523BB
:1030F0006371627973799A4203D105212000FFF749
:10310000CFFF70BD6123F3E76623F1E76B23EFE7A1
:103110007023EDE77523EBE77A23E9E73123E7E74F
:103120003223E5E773B505002E000100214A684609
:103130001136FFF7C9FF36011F4CB01C6946001954
:1031400005F02EFF14200222002168432B010019F4
:10315000A6191B197272FE330200998304250123FC
:103160004A321380C36495711381D37205008022A3
:10317000563552002A80A262104A0225A2852200FA
:103180002E32E38413702300FF355830058030332E
:103190002000197023003430017033330C220848AA
:1031A000197005F0A4FE230048340833DD8725801C
:1031B00073BDC04600920008A40000200302000076
:1031C000DE000020F0B505002E0085B00100BA4AEF
:1031D00002A81136FFF778FF3701B84CB81C001968
:1031E00002A9E719FEF7FEFA7A7A052A01D9002228
:1031F0007A72B34B32011988A2180F00507A0093EB
:10320000074101203B00034007420FD153720029C0
:103210000CD00A000240014208D10B001341D7B282
:10322000034200D1ECE13201A21857722A01A11821
:10323000FF31C87E052801D90020C876009BA1185F
:103240005888FF3107008C46C97E0F4101213B00A1
:103250000B4001930F4213D16346019FDF76002894
:103260000ED007000F4008420AD1FBB201930300C1
:103270003B410B4200D1C8E1019BA118FF31CB7645
:10328000A118FF31087F032801D9002008773601F3
:10329000A619717A012904D9042902D00021009BC2
:1032A0009980009BA1189888FF3107000E7F374155
:1032B00001263B00334037420FD10B7700280CD05A
:1032C00001003140304208D103000B41CFB23342FC
:1032D00000D19FE1A218FF32177714221100694331
:1032E00061184A310878042801D9012008706A431E
:1032F000A2184B321178042901D90021117014222F
:10330000009B6A43998EA2180B004B32107801265D
:103310000341334212D1167000290FD04810020029
:10332000324030420AD10F001741D0B2374200D1AB
:1033300075E114226A43A2184B32107014226A43BA
:10334000A2184C321178032901D9012111701422DD
:10335000009B6A43D98EA2180B004C3210780126CC
:1033600003411F003740334211D1177000290ED09E
:103370000A00324031420AD10F001741D0B2374221
:1033800000D151E114226A43A2184C321070142269
:103390006A43A2184E321178012901D90021117017
:1033A0001422009B6A43198FA2180B004E3210782A
:1033B000012603411F003740334211D11770002905
:1033C0000ED00A00324031420AD10F001741D0B26C
:1033D000374200D12DE114226A43A2184E321070F8
:1033E00014226A43A2184F321178022901D9002110
:1033F00011701422009B6A43598FA2180B004F32A0
:103400001078012603411F003740334211D1177055
:1034100000290ED00A00324031420AD10F00174174
:10342000D0B2374200D109E114226A43A2184F32C8
:10343000107014221100694361184D310878022878
:1034400001D9002008706A43A2185032117805296A
:1034500001D90421117014221100694361185231FD
:103460000878012801D9012008706A43A218553252
:103470001178012901D90121117014226A43A2187F
:1034800053321178022901D9002111701422009BB6
:103490006A43998FA2180B0053321078012603411A
:1034A0001F003740334218D11770002915D00A0089
:1034B0003240314211D105E000920008A400002002
:1034C000600200200F001741D0B2374200D1BAE0AD
:1034D00014226A43A2185332107014221100694357
:1034E0006118563108780C2801D9002008706A4309
:1034F000A21811004C310978012905D14F321178F9
:10350000022901D10021117014226A43A21810006F
:1035100001215730017002205832FF301080E21D27
:10352000D07F042800D9D17722000832D17F042926
:1035300001D90021D177009B21006C331E8808310E
:103540003700CA7F01201741874A07420FD1C87749
:10355000002E0CD0771039000140074207D133000C
:103560000B41CFB2034273D011000831CF77210055
:1035700028310878022801D900200870210029315B
:103580000878022801D901200870009B26006E33BC
:10359000188829360100337819410B0001211F00DA
:1035A0000F400B420ED1377000280BD003000B40A8
:1035B000084207D107001F41DEB20F424CD0130072
:1035C00029331E702A3423780C2B01D90023237051
:1035D0001300323319780C2901D900211970130016
:1035E0002B331978042901D9002119700023180000
:1035F0005E4900240C572600783631DA087031E035
:103600000132102A00D008E610E60137102F00D052
:103610002BE635E60131102900D055E65DE6013292
:10362000102A00D07FE689E60132102A00D0A3E6F6
:10363000ADE60132102A00D0C7E6D1E60132102AE9
:1036400000D0EBE6F5E60132102A00D03AE744E775
:103650000131102983D18AE70133102BAAD1B1E7B8
:10366000782CCBDC0133DBB201310C2BC1D1002330
:1036700001203F490C78022C00D908700133DBB2DD
:103680000131042BF6D1130034331978012901D903
:1036900000211970374B140070331888343401003E
:1036A000237819410B0001211E000E400B420ED160
:1036B000267000280BD003000B40084207D10600FB
:1036C0001E41DCB20E424AD0130034331C7013008A
:1036D0002C331978052901D90321197013002D33D2
:1036E0001978012901D90021197013002E33197896
:1036F000022901D9012119701300303319780229E8
:1037000001D9002119701300333319780C2901D91C
:103710000021197014236B43D3181800FF21513076
:103720000170C17010002F30017010002D0155196B
:103730003130017028000139FF39FC300162180076
:10374000FE355A305C3369840180198013003533AB
:10375000116291841970D186118705B0F0BD0133D3
:10376000102BACD1B3E7C046A4000020DE0000203F
:10377000EA0000206002002070B5052821D8FCF77F
:10378000D5FC2103261B2126010020251F240F2202
:10379000114B1E001A770122987003384836C0B2C8
:1037A0003580824292411D0052424A352C80197167
:1037B0009A7319749A7670BD09256F240021072227
:1037C000E6E7FEE71425322400210A22E0E735254A
:1037D000132402211922DBE748000020F0B5050080
:1037E0001135844A2D01AB1C9B1885B006001800CA
:1037F00000920193FEF718F807000421039003A834
:10380000FEF7CCFB7C4C009A2300A7606761012780
:1038100051331F70230052331F80230054331F8005
:10382000009BE0835D196B7A63703301D318FF331B
:10383000D87EFFF7A1FF009A704B0732D27F6078E5
:103840009200D35623732376052808D8FCF76EFC24
:1038500003065B5D5F610023637300E06773230011
:1038600001200222617B28331970654B61761B8829
:10387000184013424FD1A08504225F4D134202D05D
:10388000A88D0243AA851A0704D510225A48878DAD
:103890003A438285DA0604D520225748878D3A4379
:1038A00082859B0603D50823AA8D1343AB852F0081
:1038B00000232A373B70994203D10198FDF7E4FFBA
:1038C0003870009A3301D318FF331A7F2B00293345
:1038D0001A70002A0AD04B4BE98B53435B18EB83D9
:1038E000494B5343AA689B18AB606B61EB8B6B62CF
:1038F0002B0028331F78052F59D83800FCF716FC09
:103900000E585A164D4F0223A6E70423A4E70523B9
:10391000A2E70323A0E70243A285ADE7A878032826
:103920003AD8FCF703FC024B49021827631CDF77E7
:10393000220023002032303343CA43C312683800C8
:103940001A602300314A4C331A80FDF773FCFF21C3
:103950008905FDF761F9FCF7DDFD2300C0B24E33A8
:103960007F0818803B1C042F00D80523220050320A
:1039700013702300FA20483319888000FCF76AFC92
:10398000009E0234E0872C363078052826D8FCF7D4
:10399000CDFB172D2225272AFEE70227C6E7AB78A5
:1039A000022B09D0052B07D0012B07D0FEE7FEE73D
:1039B0001927BBE70627B9E70C27B7E71227B5E7B2
:1039C00096239B012A006B640023563258351380DE
:1039D0002B7005B0F0BD96231B02F3E7E123FBE754
:1039E000E1235B02EEE7E1239B02EBE79623DB0199
:1039F000E8E7C046A400002048000020C893000863
:103A0000600200201111000011111111E2040000E8
:103A1000DE2210B5FF210248520005F068FA10BD01
:103A2000A4000020DE2110B502484900FEF73CFF4B
:103A300010BDC046A4000020DE2110B50248490098
:103A4000FEF71CFF10BDC046A400002010B5FFF714
:103A5000F3FF024B1878FFF7B5FB10BD48000020BC
:103A600070B5FFF7D5FFFEF733FF04280CD0FFF742
:103A7000CFFFFEF72DFF042803D1FFF7DDFF042859
:103A800006D0FFF7C5FF03E0FFF7D6FF0428EED10D
:103A9000274E284C10223100200005F04BFA002858
:103AA00008D010222000244905F044FA002801D053
:103AB000FFF7AEFFA123A28A00259B019A420DD0F9
:103AC00008D328000135EDB2FFF72CFB0A2DF8D101
:103AD0000023E377A12301259B01A382174B2269D1
:103AE0009A4201D00125236110223100200005F007
:103AF00021FA00280CD0102231002000FDF79AFF97
:103B000008220F490F48FDF795FFFFF78BFF01E0F3
:103B1000002DFAD10023E3770B4C2370FFF77AFADC
:103B20002078FFF74FFB2078FFF758FE70BDC046A6
:103B300007920008A4000020189200084228000004
:103B400029920008560200204800002030B5C01A13
:103B500003AC12302578041C1F2800DD1F2420042C
:103B600000D5002424B2AC4200DD2CB2E4B2123BFA
:103B70000C70E418147030BD07B5080011001A006D
:103B800018230093FFF7E2FF07BD000037B50500DB
:103B9000022900D9FEE70A4809014418A37862788F
:103BA000095CEC60280004F0DDFFE07963790190A6
:103BB000A07922790090E178280004F0FBFF37BD5E
:103BC00008A90008836870B50400002B0CD003001E
:103BD000020000681432C56915332000A84720226E
:103BE0002000217D05F02FF870BD00007FB58160B9
:103BF0008D7A0400002D29D0012104F093FF0121CA
:103C0000200005F084F80121200005F097F8082134
:103C1000A36820005956FFF7D5FFA3682000197844
:103C2000FFF7B4FF00222000110004F090FF0023F2
:103C30001D4A009320001D4904F0D0FF20001B49BD
:103C400004F0ECFF200005F06BF87FBD032104F0C9
:103C500069FF2000012105F05AF82000012105F03C
:103C60006DF80821A36820005956FFF7ABFFA36841
:103C70002A005E680E4B200023618621102305F088
:103C800085F80C4B200003935B23042201937021E1
:103C9000029500954B3B05F085F82A003100200085
:103CA00005F0A8F8BEE7C04603400000FFFF000093
:103CB000F4A80008E86A000010B5040005F030F828
:103CC0002000024904F0AAFF10BDC046FFFF00001B
:103CD00070B503000400020081680068097AC569B4
:103CE00015331432200049B2A847A3689A7A002AF3
:103CF00008D01A78022A00D9FEE7044B12019B185B
:103D0000E36070BD024B2361FBE7C04608A90008D1
:103D1000F4A80008836810B50400181E0FD0E368EB
:103D2000002B05D12369002B02D12000FFF7D0FF23
:103D3000A3689B7A002B03D0E3680C20185E10BDAB
:103D400023691020185EFAE7836810B50400181E76
:103D50000AD0E368002B05D12369002B02D1200093
:103D6000FFF7B6FF1520205610BD00000300D83322
:103D70001B78002B0AD0D9300278074B1201991812
:103D80008968D2580978890088587047837D0E3336
:103D90009B001858F9E7C0466893000837B51B4ADE
:103DA00043780178D28B1B0204000B4301209A4216
:103DB0002BD12F22A3780018934326D1A379812BEE
:103DC00023D86B469D1D012321005B422800223A27
:103DD0002B80FEF7CDF8A37B617B2A881B02032092
:103DE0000B439A4211D121004C2228000D31FEF7DD
:103DF000BFF823005A3459331A78237828881B02D5
:103E00001343C01A431E984180003EBD4800002065
:103E100010B507240B7ACA7923401B021343038091
:103E20004B7A0A7A38342340D2085B01134343802B
:103E30004B7A8A7A9B0992001A43CB7A3E3C234004
:103E40009B0213438380CA7A0B7BE2400E342340EB
:103E5000DB011343C3800B7B9A060FD4302213403F
:103E60005A1E93419B0203830B7B7F2B08D83F2272
:103E700093435A1E93419B02438310BD014BF2E7CB
:103E8000004BF9E7FF070000F0B507273F250124A5
:103E90000B7ACA793B401B02134303804B7A0A7AA0
:103EA0002B40D2085B01134343804B7A8A7A9B09EB
:103EB00092001A43CB7A23409B0213430F22838044
:103EC0000B7BCE7A1340E640BB403343C3800B7C70
:103ED000CE7B3B401B02334303814B7C0E7C2B404B
:103EE000F6085B01334343814B7C8D7C9B09AD001D
:103EF0001D43CB7C23409B022B4383810B7DCC7CD9
:103F00001340BB4064082343C3814B7DDB00038225
:103F10008B7DDB004382CB7DDB0083820B7EDB006D
:103F2000C3820B7B9A0625D4302213405A1E93413C
:103F30009B0203830B7B7F2B1ED83F2293435A1E89
:103F400093419B0243830B7D9A0617D43022134082
:103F50005A1E93419B0283830B7D7F2B10D83F22F7
:103F600093435A1E93419B02C3838023DB00038447
:103F70004384F0BD034BDCE7024BE3E7014BEAE788
:103F8000004BF1E7FF07000073B5264B0126DB8BE2
:103F90000D0003701B0A43704A7808218378324071
:103FA000D2008B43134383706A79C3783240B343A2
:103FB0001343C370AA7943793240383192018B435D
:103FC00013430400437102202856FDF70DFB430004
:103FD000E078210030401843E0707F20EA782379B0
:103FE00002408343134323712A79DBB23240D2016A
:103FF0000340134323712A796379F2404038024029
:104000008343134363716B469D1D012328005B426C
:1040100059222B80FDF7ACFF2B78593423706B7835
:10402000637073BD48000020F0B585B001930AAB02
:104030001B7804000E0015001F1C522B00D95227BC
:10404000FBB25B2200212000009304F050FF072206
:10405000314B2978DB8B114023701B0A6370A378E6
:10406000360193430B430821A3706B780220DB00D9
:104070000B401E43A378383113401E43A67001261F
:104080006A79E3783240B3431343E370AA796379E2
:10409000324092018B43134363712856FDF7A4FA13
:1040A0004300E07830401843E0707F20EA782379BD
:1040B0000240834313432371297922793140C90196
:1040C00002400A43227129797B00F140A779627985
:1040D00037401F4300234038014082430A43627146
:1040E000A771E11D0098DAB2904210D802AB9D1D75
:1040F000012321005B42592228002B80FDF738FF65
:104100002B78593423706B78637005B0F0BD019A39
:10411000D25CCA540133E5E74800002007B500939C
:1041200013000A000121FFF77FFF07BD30B54D4A9C
:104130000178D31DDC7F0F231C409943214301707C
:1041400011000831CC7F017824011940214301700E
:10415000110028310C7841781C409943214341706B
:10416000110029310C784178240119402143417014
:1041700011002A310C7881781C40994321438170C9
:10418000110032310C7881791C40994321438171AF
:1041900011002B310C788178240119402143817062
:1041A000110034310C78C1791C4099432143C1710D
:1041B00011002C310C78C1781C4099432143C17007
:1041C00011002D310C78C178240119402143C170B0
:1041D00011002E310C7801791C4099432143017163
:1041E000110030310C7841791C40994321434171D1
:1041F000110033310C78817924010B402343837102
:104200000400030018490B33173400254D570131C2
:104210001D700133A342F8D11300032446331978EB
:10422000C37D2140A3430B43C37513000C254733C3
:104230001978C37D2140AB4389000B43C37513003C
:1042400048331978C37D21402D340901A3430B4322
:104250003F21C37549321278DBB292010B40134300
:10426000C37530BDA4000020DE0000200278364B6C
:104270001207120FD91D30B5CA771900027808311C
:104280001209CA771900427828311207120F0A70F2
:1042900019004278293112090A70190082782A31EE
:1042A0001207120F0A701900827932311207120FA9
:1042B0000A70190082782B3112090A701900C2792C
:1042C00034311207120F0A701900C2782C3112070C
:1042D000120F0A701900C2782D3112090A701900E4
:1042E00002792E311207120F0A701900427930310B
:1042F0001207120F0A7019008279333112090A70FD
:104300000400020011490B321734002555570132C1
:104310000D700131A242F8D11900C27D46319207D9
:10432000920F0A701900C27D47311207920F0A706E
:104330001900C27D48319206920F0A70C27D49333E
:1043400092091A7030BDC046A4000020DE00002093
:10435000F0B5522799B003AC3A0005000E002000DA
:10436000002104F0C4FD212320482370FDF748FB01
:104370006080A1208001FDF743FBA0801220142261
:104380001B496844FDF756FB1A48FFF7DDFC1A4B42
:10439000A07651331B780AA8E376FFF7C7FE802387
:1043A0005B426387154B164A1293164B28001393F2
:1043B000154B149315AB1A80144B1A006C321188EC
:1043C00056226A4411701A006E32118857226A44CC
:1043D000117070331A8816AB1A7002212300320054
:1043E0000097FFF721FE19B0F0BDC046422800003B
:1043F0002F9200085C0A0020480000206400FA00A8
:10440000FF7F0000F401E803FF7FFF7F60020020D0
:10441000010070B5040005001B3106220A48FDF7B3
:104420006BFB200019352A7A084B1207FF33120F55
:104430009A762A7A25301209DA766A7A1207120FEA
:104440001A77FFF713FF70BDB6010020A40000200B
:1044500070B50023082504000A4A8380126883711E
:1044600083810384826008492A00103004F0A0FD93
:1044700020002A000549183004F09AFD044B2360FF
:1044800070BDC046B01600203D920008469200085C
:1044900060EA000010B50220FFF76EF9104C200012
:1044A000FFF70AFC802120004942FFF78BFBA3683D
:1044B000002B00D1FEE70021200004F01DFBFA20B4
:1044C0008000FEF72FF92000012104F02BFBA368E8
:1044D00020001978FFF75AFB2000FFF7EDFB10BD15
:1044E0005C0A002070B50400451CEB7F0234002BF1
:1044F0000ED1FEF7B6F8002801D1E07770BDE37F5A
:1045000001335BB2E377312BF8DD0123EB77F5E77D
:10451000FEF7A7F8002802D03223E377EEE7E37F27
:10452000013B5BB2E377002BE8DCE877E6E70000CD
:10453000421C0C4BD27F1B68002A11D082689B1A48
:10454000FA221201934201D9012343710379002B0E
:1045500005D14379002B02D0012303710373704707
:104560008360F3E7B01600200300007B0022811E69
:10457000012903D8591CC97F914201D11A73704790
:104580001000FCE70A4A70B51388040001339BB29F
:104590000D00502B01D8138070BD002305491380F6
:1045A000FDF7E8FD29002000FDF7E4FDF4E7C04633
:1045B000380300204F920008F0B51700050085B0C1
:1045C00002916949FDF7D6FD39002800FDF7D2FDBB
:1045D0000022664B664C1A80029B012B0FD180266D
:1045E000FF33A3616348A662FEF79CF86148A661A9
:1045F000FEF798F839002800FFF7C4FFF2E7029BA6
:10460000981E80230C2800D9A1E0FBF78FFD071727
:1046100028384BA0A0A05E5E5E5E5E008026A3618F
:1046200076005448A662FEF77DF85248A661FEF770
:1046300079F839002800FFF7A5FFF2E780238026EC
:104640005B00A3624B48A662FEF76CF84948A6617E
:10465000FEF768F839002800FFF794FFF2E780269C
:10466000A36276004348A662FEF75CF84148A66163
:10467000FEF758F839002800FFF784FFF2E780269C
:1046800080237600A3623B48A662FEF74BF88023A6
:104690003848A361A661FEF745F839002800FFF706
:1046A00071FFECE7802680237600A3623148A66183
:1046B000FEF738F880232F48A361A662FEF732F890
:1046C00039002800FFF75EFFECE7029B093BDBB2F5
:1046D000039300230193019B039A934202D2802308
:1046E0005B00A362042680232248A362FEF71AF827
:1046F00080232048A361013EFEF714F8F6B239008A
:104700002800FFF73FFF002EEDD180235B00A3615F
:10471000043680231748A362FEF704F88023154867
:10472000A361013EFDF7FEFFF6B239002800FFF756
:1047300029FF002EEDD1019B0133DBB20193029BD7
:10474000019A083BDBB29342C5D20196C3E7A3624C
:1047500080235B00A3620848FDF7E4FF39002800CE
:10476000FFF710FFF7E7C0464F920008380300201C
:1047700000040048A861000050C30000F7B50D0018
:104780001E0000280DD16B46064C9F1DD91D3A0016
:10479000200004F0ADFA33002A002000397804F03C
:1047A00086F9F7BD5C0A0020F7B506000C0017007B
:1047B0000F4D0193002816D1FDF7D6FE3B002200D5
:1047C0003100280004F04EF928000A4904F026FAC6
:1047D000019B28001A01012192B204F042FA7D20C7
:1047E000FDF7A0FFF7BD2800FFF766FAFAE7C0461D
:1047F0005C0A0020FFFF0000F8B55B2705001F4C96
:104800000E003A000021200004F071FB2B7E0120F5
:1048100023706B7E00216370AB7E2173A370EB7EEF
:104820006173E3702B7F164923716B7F6371AB7FDC
:10483000A371EB7FE371134B1A78023A53425A414A
:10484000637A8343134342222000A2721A3A6372AE
:10485000E2720E30143AFDF7EDF859212000FDF711
:104860009DFB230059331870000A5870064B3A001C
:10487000300021001B7FFFF797FFF8BDE7080020FD
:104880002F9200082B03002048000020F7B50C00F1
:10489000002809D10E001348A0368368A234002BEB
:1048A00003D1812232702370F7BD9F7A6B469D1D24
:1048B000002F0DD02200290004F0F7F90022AB5E92
:1048C000002B0ADB01235B422B802B883370EBE744
:1048D000290004F0C7FA2770F0E77F33F5DA7F2369
:1048E000F1E7C0465C0A0020034B0A0010B5010046
:1048F0001800FFF761FEC0460C0000200023FF22D5
:10490000037043708370C2700371704710B5C17833
:104910000300002905D182780171013282700120E3
:104920000CE00478012C21D0022C08D00020844215
:1049300004D19A78187101329A70013010BD8078D4
:104940005A784240D20704D40022013098701A717C
:10495000E5E7FF2902D100201871EFE71A7901324B
:10496000D2B21A719142EFD30020E7E7FF29F2D0CB
:1049700002790132D2B202719142F5D282780132CB
:104980008270002202712000D8E7000010B5027882
:1049900043789A4210D0042B0FD803700278094B49
:1049A0009200D1560848094B197319768368002B79
:1049B00002D01972FFF706F910BD0423037043708B
:1049C000ECE7C046C89300085C0A002048000020BD
:1049D00010B5002A01D1437010BD541E0B2CFBD81A
:1049E0000332D2B25200515A124A91420AD95AB2F3
:1049F000111C002A00DA00214AB29A4200DD5AB2A4
:104A00004270E9E7C1225200914202D29A1E52B28C
:104A1000EEE7094A914205D959B201220329ECDC9B
:104A2000DA1EF4E7CB240022A400A142E5D35A1EEB
:104A3000EDE7C0467E060000D404000080230D4848
:104A400010B5C2691A4211D002681A420ED00A4B40
:104A50000A4A19881388994209D013880133DBB2B6
:104A600013801388064A9BB2D35C038510BDFDF703
:104A700057FAFBE700380140A40C0020A20C0020EC
:104A8000A20B00200D4902000B880D4810B5013320
:104A90000488DBB200209C420ED00A48C2540B802E
:104AA000EFF31081012080F310888023064A1468F8
:104AB0002343136081F3108810BDC046A40C00206E
:104AC000A20C0020A20B00200038014070B50400A9
:104AD0004518AC4200D170BD2078FFF7D3FF0134F8
:104AE000F7E710B508001100FFF7F0FF10BD000058
:104AF00070B50C0088B0060015000021082206A839
:104B000004F0F5F923005A1E93411B0302930C2372
:104B100001A90448019603950494059303F020FE2F
:104B200008B070BD0038014070B50125044C236801
:104B3000AB432360FFF7DCFF23681D43256070BD96
:104B40000038014010B5002908D080228021044897
:104B50009201C900FFF7E8FFFDF758FD012010BDE5
:104B6000A086010010B5002906D0002203481100DC
:104B7000FFF7DAFFFDF74AFD012010BD9A5B060042
:104B800010B5002908D08022802104489201C90074
:104B9000FFF7CAFFFDF74CFD012010BDA086010004
:104BA00037B501258020314CC0012368AB43236019
:104BB000FDF7A8F902238021902000930A225B19B7
:104BC00001958900C005FDF75DFB00222848110012
:104BD000FFF78EFF6368274AC62013402A228021F0
:104BE0006360A36880009343234AA36013580906B7
:104BF0001B021B0A0B43135080231B05136020006C
:104C0000FDF78EF9EFF3108185F3108840222368B9
:104C10009343236081F3108822620022174B802186
:104C20001A80174B89031A806368164A13400822BA
:104C30006360A3689343A3606368134A134022220E
:104C40006360A3689343A3608023A2685B0113435E
:104C5000A36023681D4380232560DB03E2690A42C9
:104C6000FCD0E2691A42F9D037BDC0460038014095
:104C7000A0860100FFB7FFFF00E100E0A20C0020CA
:104C8000A40C0020FFF7FFFFFFBFFFFF30B585B08A
:104C9000002105000E22684604F029F9184C6A46E6
:104CA0002300A0331B8820001380FCF741FC6B46D7
:104CB00098702000FCF731FC6B46D87023006A46E0
:104CC000A4331B880F489380FFF73EF86B4698711A
:104CD00023006A46A6331B786946D3712300A933A3
:104CE0001B78AA341372238828005381064B9B78C3
:104CF00013730123537302F097F805B030BDC0461B
:104D0000A00900205C0A00204800002010B50248DD
:104D1000FEF7F8F810BDC0469D090020F8B50E005A
:104D20000700204C5B232100150030002200FFF714
:104D300025FD6278237812021A43A37821791B0497
:104D40001343E27812061A4363791B020B43A179DD
:104D500009041943E3791B060B433969914202D1D7
:104D60007A699A4209D0002530000F49FFF78EFD7D
:104D70000120002D00D00230F8BD20005921FDF7A0
:104D80000DF923005A3459331A7823781B02134340
:104D90008342E8D1002D02D0FFF7B8FFE4E70125F8
:104DA000E2E7C046910A0020A009002013B50400E4
:104DB00001210130FDF7F2F86B46D880A178981DEB
:104DC000FDF7CAF86B46E178981DFDF7C5F86B460C
:104DD0002179981DFDF7C0F86B466179981DFDF7A4
:104DE000BBF86B46A179981DFDF7B6F86B4621001C
:104DF000981D03220831FDF7BBF86B46210062784D
:104E0000981D0C31FDF7B4F82423FF33E15C6B46A9
:104E1000981DFDF7A1F86B46DB88FE34E38113BDD6
:104E2000F7B51E001A4B01921A00303212780400B6
:104E30000D00002A2AD02B331B78002E05D0002B22
:104E400024D0043B5A1E9341DEB2124BE718124B9A
:104E5000E31800932888FCF749FC38802888FCF781
:104E600059FC009B3884023702359F42F2D10B4B2C
:104E7000BD211A68BC239B00E2500122084B890027
:104E8000E654019B53406354064BE254F7BDC046C1
:104E9000A4000020AE020000CE020000B0160020E8
:104EA000EE020000AD020000C423F0B59B00C6185E
:104EB000B13BFF3BC35C05009C46C42362469B009C
:104EC0006135C254FF356A782F4B85B0C2542B79B7
:104ED000040000936B792D4F0293AB792C4801931A
:104EE000AB681B021B0AD9B203916146FD293BD175
:104EF000A978E155C521EF78890027540A27009841
:104F0000605402992348215423490198605423494D
:104F1000D8B2605418120131605421491B146354F3
:104F200021006D31F019FF3104F042F86B78FF1861
:104F30001C4BB91CE218D38989B2F355D2897B1C6A
:104F40009BB2120AF254AB78DB0708D59C239B0076
:104F500070180D22E1180F3704F02AF8B9B23000AA
:104F6000FDF7F6FD05B0F0BD0023AB70009B019985
:104F7000E355029B06272354C5239B00E154039B62
:104F800004496354CCE7C04611030000120300003B
:104F900013030000150300001603000017030000B0
:104FA000190300005E020000F0B58C220700C38BDD
:104FB000060089B028375200934209D300230377B3
:104FC000CB1CDBB2012B10D90023F38309B0F0BD59
:104FD000007F0E2864D8FBF79FF8F30D202D636344
:104FE000636363636363636335000123F383397031
:104FF0003377EBE75A1CF283F9543B7889B2FD2BE7
:1050000005D1F33B0C3133847184083BF0E7062370
:105010000831338471840833EAE75A1CF283F95467
:10502000CB0702D5738C0D33738400230129DFD89D
:105030000333DDE75A1CF283F95400239942D7D198
:105040000E33D5E75A1CF283F954F28B738C9A42D3
:10505000BCD30023F38333773B780193FD2B25D119
:1050600033003200303331321B7812781B021204C5
:105070009B1832002F3212789B18A64ABC200024BD
:10508000944640000C25221801325208554329004D
:10509000654649598B420DD2501EA042F2D80CE011
:1050A00000233377F383338473848FE733002D3306
:1050B0001B78E2E714008B42EFD80C216246614373
:1050C0005258934200D081E70A230093019BFD2BA5
:1050D00001D0062300933000293003780293029A0E
:1050E000009B94466344591E89B20193FCF756FF16
:1050F00006ABD8800C236343864DED182B7919003D
:10510000049306AB981DFCF727FF019BFB185A7808
:10511000019B1202FB5C9B1806AAD2889BB29A42A2
:1051200000D053E7AB7901221900114003911342DB
:1051300009D00021EA7903910299914203D900999B
:1051400079188A5C039202221900114001911342DE
:105150000DD00A3262436F4B9B1800221B7A0192DA
:10516000029A9A4203D9009ABA18D35C01930C228E
:105170006243684B34009B185B79613402933300BF
:1051800028331D78B0235B00F554330029331B7896
:10519000FF346370009333002A33187859789A7873
:1051A00003331B780593FD2D72D163713300227197
:1051B000A070E1702E331B783200A37133003132BE
:1051C00030331B7812781B0212049B1832002F32E6
:1051D0001278F33D9B181B021B0A3200300061322B
:1051E000FF3291681B02090E09061B0A0B439360EC
:1051F0006D30009A7919FF3003F0DAFE029B009AB5
:10520000934206D9009800210C309A1A201803F016
:105210006EFE30006130FF304378EB18FA18517899
:10522000FA5C090252183C497118CA818278D20787
:1052300008D5023399B29C239B000D227918F018EF
:1052400003F0B6FE354B039AF3181A70344B019AEB
:10525000F3181A70334B049AF3181A70A123029AA8
:105260009B00F3181A70A02302229B00F3181A70F7
:10527000B4235B00F3581B021B0A6E2B3ED12A4B52
:105280009878052816D8FAF751FF343D400D344080
:10529000B12300255B00F552059B20716171A2715D
:1052A00006359AE75A6CE1239B0293429B415B428D
:1052B000002B23D0B7235B00F35C012B1ED8B9234E
:1052C0005B00F35C042B19D130007C3010221749AD
:1052D000FF3003F02FFE002810D1C42278235200A3
:1052E000B354063AB354063A2000B354FFF75EFDB8
:1052F00004E0E12252025B6C9342DBD83000FFF7FE
:10530000D3FD63E6E1221202F5E75A6C96231B02F5
:10531000CBE7C046089400085E020000810200004E
:105320008202000083020000480000205192000821
:1053300070B50A4B08002D331B781100012B0AD1E0
:1053400004008518AC4200D170BD21780448FFF7F5
:105350002BFE0134F6E7FDF7FBFBF5E7A400002088
:1053600030040020A3229200835810B501338350EB
:105370000832835801338350FDF712FC10BD000042
:1053800010B5064B2D331B78012B03D10448FFF7D2
:10539000E9FF10BDFDF704FCFBE7C046A4000020B8
:1053A00030040020A223F7B5AB25FA229B00C35896
:1053B000AD0004000E00475DCB1A9200934229D243
:1053C000632B01D80020FEBD012F0CD0022F1BD073
:1053D00000208742F7D1FDF7CDFB8023DB00984208
:1053E000F0D9012306E0FDF7C5FB8023DB009842DE
:1053F00002D9022363550DE0FDF7BCFBC0235B001F
:105400009842DFD20023F5E7FDF7B4FB8023DB00F1
:105410009842E6D3A2239B00E6503948FCF7B9F83E
:10542000384A394D1168431A01932B6859428C460A
:105430000199614501DB994259DD0A2310602B6017
:10544000FA2311685B00994200DA1360A3239B00E2
:10545000E558642310685D43123B58432B4B483397
:105460001988FAF7F7FE01002800FAF769FE00250F
:105470005F2809D81E35552806D846353B2803D95C
:10548000093D4A2800D9293DAB239B00E35C022B50
:1054900031D0012B31D0002B02D1002F00D0332589
:1054A000A522A620FA23920080009B00201831003C
:1054B000A258FCF795FCAB2300209B00E35C8342E1
:1054C0000ED1642D0CD1A2229200A35810495B1872
:1054D000A350A3239B00E05803214000FAF730FEBD
:1054E000A3239B00E05004330120E5546BE7002B1D
:1054F000A6DD013BA3E70025D2E73225D0E7C04671
:10550000A0090020FC020020080000204800002024
:1055100066FDFFFFF8B5A2239B00C358AB250E0024
:10552000CB1AFA21AD000400425D89008B4211D2F2
:105530000020032A0BD81000FAF7F8FD021E2F3BBB
:10554000FDF718FBC8239B00984201D80020F8BD46
:1055500001236355A2239B00E650394B4833198839
:10556000A3239B00E7582033E55C032D66D8280071
:10557000FAF7DCFD4A226062FDF7FCFAAF23DB009C
:10558000984201D90223E4E7FDF7F4FAA328DDD815
:10559000AB2303229B00E254DCE7632BD6D9FDF753
:1055A000E9FAAF23DB009842D4D2AB2301229B005F
:1055B000F1E700206055CAE72125A522A620FA239D
:1055C000920080009B0020183100A258FCF708FCD4
:1055D000AB2300209B00E35C83420ED1642D0CD1F1
:1055E000A2229200A35817495B18A350A3239B0043
:1055F000E05805218000FAF7A3FDA3239B00E050AB
:1056000004330120E554A2E764230F485F43FAF70F
:1056100097FD01003800FAF793FD5F28CDD81E25CD
:105620005528CAD846353B28C7D9093D4A28C4D988
:10563000293DC2E70025C0E75D25BEE76425BCE73C
:1056400048000020E0FCFFFF50400100F8B5254F66
:1056500004003800FBF756FFFBF7DBFF0600A6202F
:105660003856FBF7D6FF05003800FBF756FFA4239A
:1056700022009B00E35C6D32FF3293710A23181AFB
:10568000031C00B2167155717F2800DD7F231904B9
:1056900000D50023D371FF23200013726D226130E7
:1056A000FF30CC3B437111338371836821001B0EA3
:1056B0001B061343220083600023FC3213670A4A4F
:1056C0005531A2181370094B094AFF31E2520922E1
:1056D0000233E3181A70FCF7D7FC2000FFF7E4FB55
:1056E000F8BDC046A009002081020000820200002F
:1056F00000B9FFFFF0B503788DB00093AC23040030
:105700009B00C75A534B0022C65A0233C55A524B0C
:10571000C05A0233E35A0193504BE35A0293AF232A
:105720009B00E35A03934E4BE35A0493B0239B0030
:10573000E35A05934B4BE35A0693B1239B00E35A7C
:105740000793494BE35A0893B2239B00E35A09930A
:10575000464BE35A0A93B3239B00E35A0B93444B03
:10576000E35C9C46B62361465B00E154404BE31882
:105770005B789C46230061466D33FF335970019975
:105780009F709972090AD97202991E711973090AD8
:10579000597303999D719973090AD9730099187205
:1057A000197404993F0A9974090AD9740599360A3B
:1057B0001975090A597506992D0A9975090AD97535
:1057C0000799000A1976090ADF705E71DD71587257
:1057D0005A745976089901335976090A99760999C4
:1057E0002000D976090A19770A9961305977090A90
:1057F00099770B99FF30D9770B0A21006F31FF3170
:10580000CB7723007033FF33DA770133DA77013354
:10581000DA770133DA77FF234371BB3B8371836807
:1058200046321B0E1B0613438360124B009AE3188B
:105830001A70F822104BD201E25226220233E318EA
:105840001A701A39FCF720FC2000FFF72DFB0DB071
:10585000F0BDC046B2020000B6020000BA0200006D
:10586000BE020000C2020000C6020000CA02000020
:10587000AE020000810200008202000030B5040088
:105880002B4B91B0C1182022684603F091FB2022D7
:10589000002108A803F02BFB264BE25C0633E35CF7
:1058A000002B01D102331A43BC239B00E15C853BF2
:1058B000FF3B2578E1548533FF33E1182300487816
:1058C0006D33FF33587088789870C97820001A714A
:1058D000002276305A71DA711032D9709D716946A2
:1058E0001A72FF30303203F063FB20003323D222E0
:1058F0006130FF30437111338371836852001B0E96
:105900001B061343A02283600B4B2100E3181D707C
:105910000A4B5201E25249220233E31855311A7000
:10592000FF31FCF7B1FB2000FFF7BEFA11B030BD2C
:10593000CE020000EE0200008102000082020000A0
:10594000BE22F0B5654B9200196883580400A7B0D9
:10595000CB1A122B00D8BAE0614B81501978A020E5
:1059600002394B4259415F4EC9B23056FBF768FECF
:1059700033000390A2331B7801255BB202933300FE
:10598000A4331B78AB4200D102353300A5331B781A
:10599000012B00D09DE007331D433300AA331B7851
:1059A000012B01D10F331D43AB363378012B00D0CF
:1059B00091E01F334C481D43FEF7D8F9FBF78CFCF0
:1059C0004A49FBF729F903F05BFA4949FBF724F947
:1059D000444E01903000FBF7ABFD04903000FBF724
:1059E000B9FD3F4B002719780590022901D1A9364E
:1059F000377802394B425941A6203A4BC9B2185662
:105A0000FBF71EFE06008022002106A803F06FFAB5
:105A1000049A06AB1A71059A1D805A71039A1F7277
:105A20009A71029A5E72DA7181230F2106AA5B4293
:105A3000538193810133FF339373019B8918180AB3
:105A40000B704870180C1B0E8870CB70132106ABBE
:105A5000C918019B2578180A0B704870180C1B0E8A
:105A60008870CB70B62330215B004942E15423009B
:105A7000002220006D33FF335A70DA707230173213
:105A80001A719D70693206A9FF3003F091FA200067
:105A9000332382226130FF30437111338371836875
:105AA000FF321B0E1B0613438360124B124AE3188E
:105AB0001D70124B2100E25285220233E31855314A
:105AC0001A70FF31FCF7E0FA2000FFF7EDF927B07C
:105AD000F0BD042360E740236CE7C046B016002009
:105AE0002B030020A00900203C03002000005039B7
:105AF00000247449810200000093FFFF820200002D
:105B0000F0B5484B0500ADB047481C68FEF71CF9DE
:105B1000BF21C02289006B58444EE31A9200B34261
:105B200002D8AB5683427BD0414B6C50A854997835
:105B3000002302930193052906D83E4B4A00D35A0D
:105B400001933D4BD35A02937F230026062705ACD1
:105B5000607312202373364BA772E1722681039380
:105B60004A331B883A002380638004ABC018FBF7DC
:105B70009BFF039B3A0059780AA8FBF76DFF019B36
:105B8000294FA380029B3800E380FEF7C3F8404210
:105B9000A0763800FEF7BEF8404264223100E0767D
:105BA0000CAF13A803F0A3F93B0007CC07C307CC45
:105BB00007C3226828001A60B6232F225B005242D6
:105BC0002C78EA542B006D33FF334B3272301A714C
:105BD00039005E709C70DE706432FF3003F0E8F9CB
:105BE0002800332382226130FF30437111338371E7
:105BF0008368FF321B0E1B06134383600F4B104A52
:105C0000EB181C700F4B2900EA5285220233EB1867
:105C100055311A70FF31FCF737FA2800FFF744F9C5
:105C20002DB0F0BDB01600205C0A0020C3090000B2
:105C3000480000204E9300085A930008810200009B
:105C40000093FFFF82020000C12370B504009B0097
:105C5000C25A0433C05C214B160AE55C204BE15C60
:105C60009C3BFF3BE25423006D33FF33F63A5E70FA
:105C70005642724152009A706F2252421A71443257
:105C80005A713D329A710022D87020001D72DA716B
:105C9000597233236130FF3043711133837183684C
:105CA0004D321B0E1B06134383600E4B4232E3182A
:105CB0001D700D4BE31819700C4B2100E3181A707E
:105CC000A1239B00E318853A55311A70FF31FCF788
:105CD000DBF92000FFF7E8F870BDC04606030000BE
:105CE000070300008102000082020000830200001E
:105CF000F8B5424F424B3A002D321E681278414BA4
:105D000004001B78012A40D139002E310D78002D76
:105D100045D0022B4BD1012D38D0022D3BD0002590
:105D2000394BE25C002A07D000223037E2543B783E
:105D3000012B4ED0022B50D0002D02D02000FFF7B7
:105D400085FC324BE25C002A04D000222000E254A1
:105D5000FFF77AFFC2239B00E35C022B15D1C3231C
:105D60009B00E358F61AFA239B009E420DD9C122EC
:105D70009200A35AF62B3AD0FA2149008B4238D030
:105D80000023A352C2229200A354F8BD3100FFF7B2
:105D900009FB0500C4E73100FFF7BCFBF9E7A223CC
:105DA0009B00C6501033E018FCF714F8B8E7A221A6
:105DB00089004358FA200025F31A8000834205D356
:105DC000A4236650322115009B00E154A6239B00BA
:105DD000E9E72000FFF78EFCAEE72000FFF74EFD5D
:105DE0002000FFF7ADFD2000FFF78AFEA4E7FCF7D7
:105DF00025FB0121064B5971C2E7C046A4000020D3
:105E0000B01600202B030020AD02000001030000AB
:105E100000030020044B0380002343608360C360C1
:105E2000036143610376704700FFFFFF70B50C25E7
:105E300004002A0000211C3003F059F820005530DE
:105E40002A000021FF3003F052F8FA22194B920089
:105E50001B6800259B18613AFF3AA350A4239B00BE
:105E6000E5541C33E554203BE5500833E55004333A
:105E7000E018FBF7AFFF104B2900E5540F4B402211
:105E8000E01803F034F87D220D4B2000E554023376
:105E9000E5500433E5540433E5500433E55004334E
:105EA000E252084BE5520233E5540433E550FFF764
:105EB000B1FF70BDB0160020AD020000AE020000C0
:105EC000EE02000006030000F8B50024FCF722FCF7
:105ED000FCF704FCFCF77CFFFCF7CAFBFCF7B8FB03
:105EE000FCF738FF2149224800F05EFFFEF758FE1C
:105EF000204DFA26AC60EC602C61FCF75FFD1E4B78
:105F0000B6001C70FCF7F4FA80221C4BD2005A61D8
:105F1000FCF742FB2D34FF34013C3000A4B2FCF707
:105F200001FC002CF8D190260127F605B762144831
:105F3000FCF7F8FBB7611348FCF7F4FB2800FCF70B
:105F40000BFB2100280002F0D7FDFA208000FCF7AF
:105F5000E9FBFDF785FD0C48FCF774FF0B4B0C4883
:105F600048331988FDF722F8F8BDC046CA00002062
:105F7000700800205C0A002014000020000401408A
:105F80008813000050C30000B8080020480000201B
:105F90009D090020F7B58022174B184ED2005A6198
:105FA0003000174902F043FE0223164C208022885D
:105FB0001A4213D0144F3D79002D10D06A46063393
:105FC0000021300002F073FD3A69009B9A4203D130
:105FD0007A69019B9A4201D000232380F7BD6A466B
:105FE0002900300002F063FD084BDA8B6B461B88FA
:105FF0009A42F3D02580F1E7000401405C0A0020BA
:10600000FFFF0000200400200003002048000020C3
:106010000023034A1370034A1370034A1370704736
:1060200029040020900A0020300300200022024BA7
:106030001A70024B1A70704729040020900A002041
:106040000300407E10B5203804280FD8FAF76EF808
:10605000060E030B0F001800FEF7DAF90122054BBC
:106060001A70054B01E00122044B1A7010BDFDF7B8
:10607000EDFCF3E729040020900A00203003002003
:1060800010B5034B1B78012B01D1FEF761F910BD50
:1060900029040020F0B53F4E9BB000903000FEF781
:1060A00035FC00240190A0421FD03B4B1C78002CF3
:1060B0005BD13A4B3A4F1B78022B52D12500380066
:1060C000ECB2FBF7ACFF002808D03800FFF758F916
:1060D00005AB58550135522DF1D12C003148A1B2F4
:1060E000FBF774FE3048FBF76BFE304D009A2B0037
:1060F000A5331A70B37802AA1370130001225A70E4
:106100002B00A4331B7802AA53711300009A2800B5
:106110009A71FBF7F7F902AB98702800FBF708FAC1
:1061200002ABD8702800FBF715FA02AB1871019B7F
:106130001F4F002B1FD0184B1E481B78002B16D169
:10614000230005AA02A9FDF7E9FF012328003B70FF
:10615000FBF712FA2800FBF71CFA0123F3701BB0BF
:10616000F0BD3800FBF7E4FFBFE70024BDE702A95C
:10617000FFF786FFE9E73B78002B00D1FEE70D48EB
:1061800002A9FDF701FF012328003B70FBF7FBF993
:10619000E0E7C046740A0020900A00202B0300208C
:1061A00018000020040A0020DC090020A0090020BB
:1061B000F80200204209002070B5294DCB782A0052
:1061C000DB07DB0FAA3213702A004B79AB325B0678
:1061D000DB0F13700600C8780C004008FBF712FABA
:1061E0002B002A00A63318702379A732DB07DB0FB8
:1061F00013702A003F212379A8325B069B0E13708F
:10620000637922790B40D2095B001343A935210041
:1062100014482B70002E02D1FDF7FAFD70BDFDF77A
:1062200033FE0F22A3789343202B03D12000FFF7E6
:1062300007FFF3E7FFF7FAFE0B4B1B78022BEDD1BC
:106240002100A279094852081931FFF771F8A179A4
:1062500007484908FBF7BAFD0648FBF7B1FDDDE743
:10626000A0090020C00800202B03002018000020F7
:10627000180A0020F009002070B5061E0BD1194B3A
:1062800019491C7819480379002B08D0012C01D03A
:10629000FBF7CCFE70BD164B16491C78F2E7164A88
:1062A000164D012C14D98B78E01E1B07DB0F5370A1
:1062B0000223137043425841C0B2FFF77DFF28000C
:1062C000FBF716F9032C05D12800FBF716F901E0BE
:1062D000012313702B002800A4331E70FBF704F970
:1062E000D8E7C04626040020EC0A00200003002066
:1062F00027040020470B0020740A0020A00900207A
:1063000010B5040009480379002B03D02100FEF7E3
:1063100073FA10BD2000FFF7BDFE054B5B22200085
:106320001B7F0449FEF740FAF3E7C0460003002054
:106330004800002042090020F8B5050026480F005B
:106340000379002B06D00A002900FEF7E7FC0400C1
:106350002000F8BD214E224C28005B232200310092
:10636000FEF70CFA3000002D00D02000FDF716FDDE
:10637000041E23D01B4E1C493000FBF7FBFE2900F6
:1063800030313000C9B2FBF7EBFE18493000FBF7A3
:10639000F1FE200002F0A2FA01003000FBF7EAFE55
:1063A0000A213000FBF7DCFE012CD1D0042C10D0E8
:1063B000012428000E49FEF769FAC9E7002F06D02C
:1063C0000C48FCF79FFD002C01D00224F1E70324C8
:1063D000EFE7002FF9D0F3E700030020EC0A0020DC
:1063E000470B00200C000020629200086992000810
:1063F000A00900209D090020034B18780238434271
:106400005841C0B27047C0462B030020F0B5A64BE0
:1064100089B01B78012B00D9FEE0002B01D1FCF7DD
:1064200051F8FFF751FDA14FA148796CFCF7FEFB35
:10643000002207249F4B1A809A709F4B80329A61EA
:10644000013CFCF73DF9E4B29C48FCF76BF9002CE9
:10645000F6D19B4D280002F089FC9A4B013880B29E
:10646000984203D901209849FEF73EFA974B391D0F
:106470001C80974B28001C80FDF7B8FB7D20FCF7A3
:1064800051F9FCF7B9F89348FDF7E2FF7B1CDB7F7D
:106490000393202B00D9FEE73B00BA8D28331B78ED
:1064A00007923A0029321278796A02923A002A3227
:1064B00012789446884A9371052B00D9FEE78748E5
:1064C0001D012E58002E00D1FEE740190579966077
:1064D000D57104958568007B1561107305901000D7
:1064E000D93003709482200022000694079D012673
:1064F0001541354205D0350095402843012580B22D
:1065000006950132062AF1D1069D734A002D00D06E
:106510009082928A002A00D1FEE7049A0598039D92
:10652000101A021CC0B2A84201D96A46127B6A4DF9
:10653000D0B2EA75052B00D198E0012B00D99EE07E
:10654000029A013AD2B2012B00D187E06346022AB7
:1065500000D97EE0013B032B74D80C230C2876D89D
:10656000EB7D029C834200D9E87563462200280037
:10657000FBF754FB2B000024FF26D8331C70584B2C
:106580002800AC751E705E70FDF7F0FB4C4D0100ED
:10659000280002F0D0FA534B1C70534B1C70534B25
:1065A0001C80534B1C70534B1C70534B1C70534B33
:1065B0001C70534B1C70534B1C70FFF729FD3A00A5
:1065C000514B02371C70514B4A321C70504B514892
:1065D0001C70F98F504B12881B88C9B2FAF74CFF18
:1065E0004D4B4E481988FBF79BFA4D48FEF786F94C
:1065F0004C4B4D482933197800F0E3FB4B48FFF72B
:1066000015FC2800FDF7A0FB494B1C80494B1C8062
:10661000FCF7AAFB244B1E70FCF7B0FB002800D14E
:10662000A9E0324A1388002B01D0013B13802E4B86
:10663000204918780B88022825D1002B31D0013B46
:106640009AB223E000239C46122889D91233EB75B5
:1066500086E7042B89D900239C4686E7022A03D8C3
:106660000C230C2809D8029C00237FE7029B013BE6
:10667000022BF9D80828F6D90823EB75F3E7280090
:10668000FBF76AFA76E7C722002BD8D18B780A800D
:10669000002B51D0002A59D1FCF704F8FCF710F870
:1066A00054E0F422FF32F1E7E40800204800002023
:1066B00010000020220400200004004850C3000005
:1066C0005C0A0020FDFF00006B9200081E04002001
:1066D00020040020000300203C03002068930008F1
:1066E000E5080020280400202B0300202E030020B2
:1066F0002C03002028030020290300202A03002067
:106700002704002026040020330300203203002049
:106710001C040020A0090020900000207C0A00201A
:10672000740A0020A400002070080020300400201B
:106730008C0A00208E0A0020B74C022800D0C7E047
:10674000002A01D1FBF7AEFF8023A361B34C23885D
:10675000002B00D1C3E0013B9BB2B1482380FDF781
:10676000C1FEB048FDF7F0FA2388002B03D1AE49F3
:10677000AE48FBF7FFFCAE4CAE4D2278002A00D1AC
:10678000AFE0022A00D1D9E02B88002B1FD023785C
:10679000032B00D0E0E02B88DB0702D500232B8001
:1067A00023702B88002B12D02B885B0400D52B88FC
:1067B0002B889B0700D52B882B88DB0700D52B88DF
:1067C00000239D4A2B8013709C4A237013709C4BAE
:1067D0001A78D6B2002A00D1E2E100201870974B57
:1067E0001F787B1E5A425341DBB20293874200D18D
:1067F000C5E0FFF741FD0023924D934A29781372BB
:10680000012900D9DCE0012F00D8BFE08F48030048
:10681000A8331B783E2B00D9BFE0A7308C4A007804
:10682000977D002800D0C4E0BB4200D1B0E0D17D0C
:106830009375994200D8A6E0029600262B78002B8B
:1068400000D02CE2029A002A00D023708149824BAA
:106850000A784E330132D2B20A7018887C4B8242D9
:106860000ADB9A7DD87D0132D2B282428041024059
:106870009A7500220A7022701A00D8321278002A03
:1068800000D104E119001800DC310A88DA30013245
:1068900092B20A800088904200D9F8E000220A8073
:1068A0001A00998AD9321278029106210132D2B2A5
:1068B000052A00D90022029F01201741074200D17A
:1068C000E0E0664910014158002900D09FE0FEE752
:1068D00080235B00A361002A00D037E7DEE6604B2F
:1068E0003BE7584B5A481B78002B07D0837DC17D6E
:1068F0000133DBB28375994200D88275FDF736FA11
:10690000484E0100300002F016F9FBF739FE300066
:10691000544902F083F900220121300002F0B3F95A
:106920007D20FBF7FFFE012323700023424A1370F2
:10693000424A13704C4A13802B8025E74B48FEF7E0
:1069400025F8414B187AFFF7DBFC03230022237064
:10695000454B1A802A8017E7012B00D021E72B88AE
:106960009B0700D41DE7344B0020197828804B4248
:106970005941C9B2FFF7E0FC304B187011E7012212
:106980003B4B1A7037E70023029693751E0055E7BC
:106990000122384807783A430270374A002919D152
:1069A0000120117028703E2B00D90331314B197032
:1069B00008E0BB4200D03AE72E4802220778EAE717
:1069C000012FE3D9244A2D4B4C3212881A8002231E
:1069D000237033E713782A4801330778DBB20521A7
:1069E0001370002F02D11C49503109789942E9D81F
:1069F000204B1B78032B04D102232B70013B037027
:106A0000E0E74B1EDBB213709942F5D9DAE7D933D0
:106A10001A70002323703AE0000400488C0A00201A
:106A2000000300205C0A0020759200080C00002082
:106A30002804002020040020270400202604002031
:106A4000310300202B0300207C0A0020A009002035
:106A50003C03002029030020480000206893000820
:106A6000E7030000FFFF00001E040020E5080020EF
:106A7000740A0020280300202C0300202E0300208D
:106A80002A0300200139C9B2002900D00EE70022F4
:106A9000874B1A702A78002A00D1FAE0002E03D121
:106AA00001221A70022323708248FDF705F92B7822
:106AB000022B02D00022804B1A70804A1388002BD0
:106AC00002D17F4B4A331B88013B9BB27D4E138022
:106AD000002B02D13000FAF76AFD3000FAF703FD0F
:106AE0002B78022B0CD03000FAF7ACFC2B78002B63
:106AF00006D1FFF79BFA0122734B1A70734B1A7081
:106B0000734E3000FCF788F97378724F012B02D175
:106B100000227B7172703800FDF70AFD3800FDF726
:106B200023FD0600012806D002282AD005226A4B40
:106B30001A7009B0F0BD3800FDF7ACFC6422604F5C
:106B4000664B4837398866484A431A80FCF7DAF9B9
:106B50003988644F64483B00D8331E70F9F77AFBDC
:106B60003B008021DA3318800023604A4900DC377B
:106B70003B809162803991615D4A2B7096702370E1
:106B8000D4E7584BD9331978052908D8594A5A4BB4
:106B9000525CFF339A760122584B1A70C6E7FEE723
:106BA0004D49574A0B78574C002B04D0013BDBB2C0
:106BB0000B70002B02D01378002B35D04E4F0025E0
:106BC0003B00157028331978200000F028F94E4B4F
:106BD0001B78022B40D1364B3A4E02931B78300083
:106BE0000393FAF78FFC04903000FAF7A1FC474EAC
:106BF000049B3100039A0190009320002B0000F0C9
:106C000091FB2000FEF742F82100029B40481A78D1
:106C100024312B00FEF704F9FB1D33373100DB7FF5
:106C20003A783C48FDF7D4FE200000F095FC384847
:106C3000FFF75EF8314B1B78002B00D179E71D4838
:106C4000FDF73AF88022294B9A6292189A62FCF773
:106C5000E9FE0122304B6BE7304B1B78002B13D041
:106C60007F235B42009380331A002849200001955E
:106C700000F058FB200000F0E5F821000123244833
:106C80001A002431FEF7CCF8FB1D224ADB7F53703B
:106C9000CAE702222378934300D105E70AE7204B95
:106CA0001B88002B00D0F2E61E4A2B701370B1E651
:106CB0001C0400205C0A0020740A00208E0A0020B8
:106CC00048000020A009002029040020900A00208C
:106CD000B8080020000300203303002044000020F7
:106CE0009D0900203C030020881300000004004898
:106CF0002204002048930008A40000203003002054
:106D000032030020700800202B030020C008002060
:106D100030040020E5080020E40800202A030020B9
:106D20002E0300202903002010B5FFF76FFBFCE7BE
:106D30000B4B0C4A10B51A600B4B0C4A0C4C1A60EA
:106D40005A619A62DA631A650A4A20005A669A679B
:106D5000094A8C331A6000F01BF8084B236010BD01
:106D60005C0A002080920008A0090020FC91000825
:106D700070080020E4910008F091000808930008D2
:106D800070470020704700207047002070470000C7
:106D900010B50400034B012108C0FAF703FB2000E3
:106DA00010BDC04644A9000870B5FF230D000021A6
:106DB0000400036181822422243002F098F8E56007
:106DC00070BD70B50D00017C0400A94218D00129E6
:106DD0001BD0022915D0002903D103685B6820006D
:106DE0009847002325746374012D14D0022D0FD011
:106DF0009D4205D123685B6801212000984760749B
:106E000070BD0368DB680021E9E703689B68FAE767
:106E10002368DB68F0E7236829009B68EDE710B57D
:106E20000430FAF7CCFA10BD10B5037C0400012B36
:106E300006D10E22163002F0BBF80223FF33638224
:106E400010BD0000037C012B0AD1064B8122C382B6
:106E500000238361038402231202FF33C261438251
:106E60007047C0468181FFFFF0B58DB00190088862
:106E70000D0002920393FAF723FC072604AB5C1D76
:106E800063782070000A3040B3430343637068881E
:106E9000FAF716FC1F223F2763780240D2003340E6
:106EA00013436370A37840093840BB430343A37086
:106EB000A888FAF705FC0323012103409A01A3786F
:106EC00078363B401343A3708308E3702379800A2C
:106ED00008408B4303432371E8880F00FAF7F0FB67
:106EE000030033401A00BA402379C0093B401343E2
:106EF000237163790E373840BB430343637128899C
:106F0000FAF7DEFB03003B401A01637900093B40BE
:106F100013436371A3793040B3430343A37168897A
:106F2000FAF7CEFB01230340DA01A3793340134380
:106F3000A3714308E37103231900400A1840237A20
:106F40008B4303432372A889FAF7BAFB3F2303213B
:106F500003409A00237A80090B40134323721F23B6
:106F600019001840637A8B4303436372E889FAF788
:106F7000A7FB07231F2103405A01637AC0080B4077
:106F800013436372A072288AFAF79AFB0722237BC5
:106F9000E072000A1040934303432373688AFAF7B0
:106FA0008FFB1F2307210340DA00237B40090B409E
:106FB00013433F222373637B104093430343637364
:106FC000A88AFAF77DFB03233F2103409A01637BE4
:106FD0000B401343012263738308A373E37B800A8E
:106FE000104093430343E373E88AFAF769FB030015
:106FF000012133405A00E37BC0090B401343E37384
:10700000237C3840BB4303432374288BFAF758FB97
:107010000200237C3A4012013B4013432374637CFB
:1070200000093040B34303436374688BFAF748FBAD
:107030000123627C03403240DB0113436374430845
:10704000A374E37C7C3E400A3040B3430343E374C3
:10705000A88BFAF735FB3F23E27C034032409B00CC
:107060001343E374237D1C3680093040B34303434C
:107070002375E88BFAF724FB0723227D0340324077
:107080005B011343C008237560752B8C104A698C13
:107090009A429B415B42914201D902221343029AD8
:1070A000002A01D004221343039A002A01D00822A7
:1070B000134305A9CB7500230F220B76019B0A70A1
:1070C0001B6801981B680A3298470DB0F0BDC04696
:1070D000A9050000F0B58BB0019008880D00FAF703
:1070E00001FB072602ABDC1D63782070000A3040EC
:1070F000B343034363706888FAF7F4FA1F223F270B
:1071000063780240D200334013436370A378400990
:107110003840BB430343A370A888FAF7E3FA03237C
:10712000012103409A01A37878363B401343A370B2
:107130008308E3702379800A08408B43034323715B
:10714000E8880F00FAF7CEFA030033401A00BA407D
:107150002379C0093B401343237163790E373840CC
:10716000BB43034363712889FAF7BCFA03003B4031
:107170001A01637900093B4013436371A3793040DE
:10718000B3430343A3716889FAF7ACFA01230340C0
:10719000DA01A37933401343A3714308E371032356
:1071A0001900400A1840237A8B4303432372A889AD
:1071B000FAF798FA3F23032103409A00237A8009C3
:1071C0000B40134323721F2319001840637A8B432B
:1071D00003436372E889FAF785FA07231F21034006
:1071E0005A01637AC0080B4013436372A072288A65
:1071F000FAF778FA0722237BE072000A10409343E3
:1072000003432373688AFAF76DFA1F2307210340AB
:10721000DA00237B40090B4013433F222373637B37
:107220001040934303436373A88AFAF75BFA03237E
:107230003F2103409A01637B0B4013430122637398
:107240008308A373E37B800A104093430343E373F3
:10725000E88AFAF747FA0300012133405A00E37B3A
:10726000C0090B401343E373237C3840BB43034303
:107270002374288BFAF736FA0200237C3A40120175
:107280003B4013432374637C00093040B343034302
:107290006374688BFAF726FA0123627C034032405C
:1072A000DB01134363744308A374E37C7C3E400A10
:1072B0003040B3430343E374A88BFAF713FA3F2338
:1072C000E27C034032409B001343E374237D1C3671
:1072D00080093040B34303432375E88BFAF702FA81
:1072E000039B0F4A1B0E1B06134303930723227DA8
:1072F000034032405B0113432375C00802AB607545
:10730000991D17220020FAF743FA02AB5877019B28
:107310001A221B6801981B6803A998470BB0F0BD9F
:10732000C8181600F0B50600040087B001930CAB36
:107330001B7824365BB204930DAB1B7802923000AD
:107340002422271D059301F033FE38003100FAF79F
:107350005FF8E568019B6879002B0CD004280AD8F7
:10736000F8F7E4FE348036680300424B6362A362A0
:10737000002301930293E3681D796B1E0B2B08D841
:107380000498FAF76BF90435EDB20F356D00651905
:10739000A880E3681D7B6B1E0B2B08D80598FAF7B5
:1073A0007BF90435EDB20F356D006519A880637C5B
:1073B000002B0BD0237C012B4FD00222934305D10D
:1073C00031002000019B029AFFF74EFD07B0F0BD8F
:1073D0002300243300932B002F0020331437039312
:1073E0000023FB5678219802C01AF8F733FF802358
:1073F000DB00C018009B0137188002330093039B09
:107400009F42EDD12A00210020323C3124351378EF
:107410000120002B08D0023B584243415B429B05B0
:10742000980D8023DB00C01801320880023195429C
:10743000EDD1A0E72200802133004832C900198035
:1074400002339342FBD102213800F9F7F7FF002302
:1074500010304000201883808DE731002000FFF7B6
:1074600039FEB3E7042800D985E70223984300D109
:1074700081E7E8E70004000430B54B7B05000C0011
:1074800085B0032B3CD100200856FAF779F96B46FA
:10749000D87001202056FAF773F96B466A461871C6
:1074A000A3785371E37893712379D371207BFAF732
:1074B0005DF96B46187206202056FAF739F96B46CB
:1074C000587207202056FAF75BF96B466A469872A5
:1074D000237A0020D372637A1373104B1380142322
:1074E00093706B460B22991CFAF752F96B4658734E
:1074F0002B680E22694628001B68984705B030BDEE
:10750000022B03D16A46FD33D370C2E70020085630
:10751000FAF736F96B46D870FF20BEE7C80C0000BA
:1075200010B5837C0400002B07D0FBF74BFCE37CF9
:10753000002B03D00023A082E37410BDA28A801A1E
:10754000FA2280B212019042F7D921002000A374E0
:107550001631FFF791FFF0E7437C10B5002B04D004
:10756000037C012B01D1FFF7DBFF10BD30B593B0D9
:107570002C22002107A801F0BAFC1022002101A84A
:1075800001F0B5FC80235B020F93802301240225C8
:107590001B0305A8059406940E95109300F026FA97
:1075A000002801D072B6FEE7072303900490210063
:1075B00001A80193029500F0A7FC002801D072B643
:1075C000FEE713B030BD000007B500F09DF8FFF7EF
:1075D000CDFF80210A4BC9035A690A435A615A698F
:1075E0000A4080210192019A5A6989020A435A612C
:1075F0005B690B400093009BFFF796FB0EBDC046F6
:107600000010024001210A4B82B09A690A439A6134
:107610009A690A4080210092009ADA6949050A4372
:10762000DA61DB690B400193019B02B07047C046F1
:1076300000100240FEE7FEE77047704710B5FBF709
:10764000ADFB10BD704700000D488546FFF7FAFFFF
:107650000C480D490D4A002302E0D458C4500433AD
:10766000C4188C42F9D30A4A0A4C002301E0136083
:107670000432A242FBD301F06FFCFFF7A5FFFEE747
:1076800000400020000000202800002098A90008E9
:1076900028000020F8160020FEE77047012210B5F0
:1076A0000024064B52421A611C61DA60DC609A6267
:1076B0009C62FFF7F2FF200010BDC04600100240A0
:1076C00070B50500FA200D4B80001978F8F738FDE9
:1076D0000B4C01002068F8F733FD00F055F804006A
:1076E0000120002C09D1032D07D8023822002900DF
:1076F00000F020F82000034B1D6070BD200000202A
:107700001C000020240000201023064A10B5116838
:1077100003200B431360FFF7D3FFFFF773FF002035
:1077200010BDC04600200240014B18687047C0469B
:10773000B016002030B5FF2503242A000440E400E1
:10774000A24089012940D243A140C3B200280ADBEC
:10775000C0240B4B80088000C018A40003591340BC
:107760000B43035130BD0F200340083B05489B08E5
:107770009B001B18D86902400A43DA61F2E7C04651
:1077800000E100E000ED00E08022431E52040120F1
:1077900093420DD2C021074A07485360036A090685
:1077A0001B021B0A0B430362002007239060136037
:1077B0007047C04610E000E000ED00E00C4A1021E8
:1077C000D06830B503000B40084205D002230948B9
:1077D000C4692343C3610B000420D168014205D072
:1077E0000121044C0343E5692943E161D36030BDC5
:1077F00000200240B8160020064B00201A6912062D
:1078000006D5054A5A60054A5A6018690006C00F35
:107810007047C0460020024023016745AB89EFCD89
:107820008023034A002011690B4313617047C0464F
:107830000020024070B50400FFF776FF0126050026
:10784000104BDA68324211D12022D968114200D09F
:10785000DA60D968102208001040114202D1DB68BA
:107860005B0708D5FFF7AAFF012004E0621CE8D0FF
:10787000002C01D1032070BDFFF756FF401BA04232
:10788000DED9F7E700200240F0B585B003931D4B29
:10789000009102921A7E04000220012A30D00122B7
:1078A00019481A76FFF7C6FF002826D12600012CBA
:1078B00002D0022C00D004260024124B019302981F
:1078C00003992201F8F7B2FD00220127019B0F4D19
:1078D000DA612B69009A3B432B6163009B1880B2ED
:1078E00018800948FFF7A6FF2B69BB432B610028CE
:1078F00003D1E419E3B29E42E1D80022014B1A768B
:1079000005B0F0BDB816002050C3000000200240B2
:107910000022064BDA61064B043219690A431A61E8
:10792000402219690A431A617047C046B816002000
:10793000002002400022064BDA61064B0232196930
:107940000A431A614022586119690A431A61704753
:10795000B816002000200240F8B5214F04003B7EFD
:107960000E000220012B0CD001233B7623681D481A
:10797000012B12D1FFF75EFF002803D00120002366
:107980003B76F8BDFFF7C4FF1648FFF753FF04210D
:10799000154A13698B431361F1E7FFF74BFF00288A
:1079A000ECD101235B42336065680130A3686268F3
:1079B000DB029B18AB42E2D92800FFF7BBFF094866
:1079C000FFF738FF0221084A13698B43136100282F
:1079D00001D03560D3E780231B01ED18E6E7C046F0
:1079E000B816002050C3000000200240F0B504008B
:1079F00085B000284ED00368DB0733D423689B078B
:107A000000D58AE023681B0700D5CAE023685B071E
:107A100000D5EDE02368DB061AD562690423BB4D6F
:107A2000012A00D056E1696B02270B436B636B6B35
:107A30001A436A63FFF778FE06006B6B3B4200D186
:107A400041E1F8216A6BA3698A43DB0013436B634E
:107A500023689B0600D565E1636A002B00D0A4E192
:107A600000202FE00C22A94D6B681340042B0BD093
:107A70006B681340082B0FD1C0226B685202134071
:107A800080225202934207D12B689B03B6D56368CC
:107A9000002BB3D1012015E06368012B14D18023A2
:107AA0002A685B0213432B60FFF73EFE8027060027
:107AB000BF022B683B42A1D1FFF736FE801B642832
:107AC000F7D9032005B0F0BD002B16D12B68904AE2
:107AD000802713402B602B688E4ABF0213402B6017
:107AE000FFF722FE06002B683B4200D186E7FFF736
:107AF0001BFE801B6428F6D9E3E7052B05D1802304
:107B00002A68DB0213432B60C9E72B68804A1340C5
:107B10002B602B687F4A1340C5E70C227B4D6B68B6
:107B200013420BD06B681340082B15D1C0226B6831
:107B3000520213408022120293420DD12B689B0700
:107B400002D5E368012BA5D1F8212A6823698A436D
:107B5000DB0013432B6055E7E2680123002A0FD0B6
:107B60002A68022713432B60FFF7DEFD06002B680F
:107B70003B42E9D1FFF7D8FD801B0228F7D9A0E7E7
:107B80002A6802279A432A60FFF7CEFD06002B6879
:107B90003B4200D136E7FFF7C7FD801B0228F6D92C
:107BA0008FE7E2690123594D002A10D06A6A022743
:107BB00013436B62FFF7B8FD06006B6A3B4200D0CF
:107BC00024E7FFF7B1FD801B0228F6D979E76A6A3E
:107BD00002279A436A62FFF7A7FD06006B6A3B42E1
:107BE00000D113E7FFF7A0FD801B0228F6D968E754
:107BF00080220021454D5205EB690091134208D1C6
:107C0000EB691343EB61EB6913400393039B01237F
:107C100000938027404E7F0033683B4215D0A36815
:107C2000012B22D12A6A13432B62FFF77DFD022725
:107C300006002B6A3B423FD0009B012B00D0E9E6B7
:107C4000EB69364A1340EB61E4E633683B4333604B
:107C5000FFF76AFD019033683B42E0D1FFF764FD16
:107C6000019BC01A6428F6D92BE70122002B14D1FE
:107C70002B6A022793432B622B6A033293432B62B6
:107C8000FFF752FD06002B6A3B42D5D0FFF74CFDB3
:107C9000234B801B9842F6D913E7052B05D1296A9F
:107CA000013B0B432B622B6ABDE72B6A93430422F3
:107CB0002B622B6A9343B7E7FFF736FD184B801B07
:107CC0009842B6D9FDE6FFF72FFD801B022800D8A9
:107CD000B3E6F6E6053203D16A6B9A436A63B0E60F
:107CE0006A6B0227134301226B636B6B93436B63D5
:107CF000FFF71AFD06006B6B3B4200D1A8E6FFF7C9
:107D000013FD801B0228F6D9DBE6C04600100240B6
:107D1000FFFFFEFFFFFFFBFF00700040FFFFFFEFD4
:107D2000881300000C22554D6B681340934209D014
:107D30006B681340082B0ED1C0226B6852021340AF
:107D4000934208D16B6B9B0300D485E6236A012B19
:107D500000D09FE680E6236A002B13D080236A6B55
:107D60005B0213436B63FFF7DFFC80270600BF0253
:107D70006B6B3B4200D06FE6FFF7D6FC801B0228FE
:107D8000F6D99EE66B6B3E4A802713406B63FFF784
:107D9000CBFC0600BF026B6B3B4200D15CE6FFF7F9
:107DA000C3FC801B0228F6D98BE60C21334D6A6890
:107DB0000A40082A47D0334A022B32D12B68802749
:107DC00013402B60FFF7B0FC0600BF042B683B425A
:107DD00021D10F22EB6A80269343226BB604134312
:107DE000EB62A16AE36A6A680B4327490A401343BE
:107DF0006B6080232A685B0413432B60FFF794FCBD
:107E000004002B68334200D02AE6FFF78DFC001BEC
:107E10000228F6D955E6FFF787FC801B0228D5D942
:107E20004FE62B68802613402B60FFF77DFC040093
:107E3000B6042B68334200D112E6FFF775FC001B35
:107E40000228F6D93DE6012B00D123E6C0216B685C
:107E5000A06A4902EA6A1940814200D01AE60F215D
:107E60000A40216B8A4200D014E6F02292031340AC
:107E7000E26A934200D1F3E50CE6C04600100240EE
:107E8000FFFFFEFFFFFFFFFEFF7FC2FF0C2070B56C
:107E9000164D6B68184008280AD00C2823D00438E7
:107EA000431E9841124B40421840124BC01870BDFF
:107EB0000F2011499A0C02408C5CEA6A0F4902407B
:107EC000895CC0228020520213404002834204D1C8
:107ED0000848F8F735F96043E9E7934201D10848CB
:107EE000F7E70848F5E70648E1E7C046001002401A
:107EF00000F7C2FF001BB7006CA900087CA90008AE
:107F0000006CDC0200127A00F7B504000F000028B4
:107F100001D10120FEBD01223A4D2B6813408B4256
:107F20001CD32268930722D4D2072FD401232A68B6
:107F30001A40BA4257D82368334D5B075AD4FFF72B
:107F4000A5FF6B68314A1B061B0FD35C3049D84034
:107F500008600320FFF7B4FB0020DBE72B689343A6
:107F60000B432B602B6813408B42D2D1D9E72649B3
:107F7000530704D5E0234868DB0003434B60F0203F
:107F80004B688343A06803434B60CDE762681E4E95
:107F9000012A03D133689B0305D4BAE7022A1AD118
:107FA00033689B01B5D5032173688B43134373601A
:107FB000FFF7BAFB01900C2372681A4063689B00BC
:107FC0009A42B3D0FFF7B0FB019BC01A114B984205
:107FD000F1D903209EE7032A01D1736BDBE73368F5
:107FE0009B07E0D495E72A689A432A602A681A42D8
:107FF000A1D08EE76B68084A1340E26813436B60B8
:108000009DE7C046002002400010024054A900082D
:108010001C00002088130000FFF8FFFF90220300DF
:10802000D20590420BD18022234B9202996A0A43D7
:108030009A629A6A214900200A409A627047204A4F
:10804000904208D180221C4BD202996A0A439A625C
:108050009A6A1C49EFE71C4A904208D18022164BCD
:108060001203996A0A439A629A6A1849E3E7184A1E
:10807000904208D18022104B5203996A0A439A62B7
:108080009A6A1449D7E7144A904208D180220A4BD1
:108090009203996A0A439A629A6A1049CBE7104A96
:1080A00001209342CAD18022034BD203996A0A432A
:1080B0009A629A6A0B49BEE700100240FFFFFDFF7B
:1080C00000040048FFFFFBFF00080048FFFFF7FF28
:1080D000000C0048FFFFEFFF00100048FFFFDFFF2C
:1080E00000140048FFFFBFFFF7B5030000220C6833
:1080F00000922000009AD04000D1FEBD0120009ADD
:10810000904022000240044231D04868032501908B
:10811000100050434543019EED43771E012F0BD8BD
:108120008F689E6847432E4037439F605F68CE68E4
:10813000A743744327435F600C69DF6844432F40C3
:108140003C43DC60019C022C0BD14F69FF2A11D803
:1081500004000F26444366437C431A6AB243224319
:108160001A62019C1A6860432A4002431A60009A0E
:108170000132BCE70F26120A52435243564357437B
:108180005C6AB4433C435C62EBE700000122294B8C
:1081900082B019680A431A60022219681142FCD0A1
:1081A000F82219689143783A0A431A600122524230
:1081B0000192019A20490A400192019A5A600C22C8
:1081C00059681142FCD11A681C490192019A0A406F
:1081D0000192019A1A6080229204196808001040E6
:1081E0001142FAD11A6816490A401A605860586359
:1081F0005A6B14490A405A63F822596B9143783AF2
:108200000A4301215A635A6B8A435A635A6B0331FA
:108210008A435A63FF221204D86218630192019ABA
:108220009A6080229860596A52040A435A6202B0E6
:108230007047C046001002400CF8FFF0FFFFF6FE4A
:10824000FFFFFBFFFFFFFEFF034B044A5B681B06BB
:108250001B0FD35CD84070470010024054A900089F
:10826000034B044A5B685B055B0FD35CD8407047E7
:108270000010024064A90008C022104B5202586846
:1082800070B5104080225202904214D00C4A8018DF
:10829000421E90410B4A404210400B4A80180F2565
:1082A000D96A5C6829400131F7F74AFFA40C2C40D9
:1082B0000234604370BD0548F1E7C046001002403B
:1082C0000080FEFF00A69DFD006CDC02001BB700D5
:1082D0000B4B10B558680C23184008280AD0984258
:1082E0000BD00438431E9841064B40421840064BC1
:1082F000C01810BDFFF7C0FFFBE70448F9E7C04610
:108300000010024000F7C2FF001BB700006CDC0247
:1083100010B50400FFF7DCFF2060FFF795FF6060F9
:10832000FFF79EFFA06010BD030010B500280CD120
:1083300003211A4A136B0B40022B29D08B421FD00A
:10834000012B16D1FFF7C4FF10BD0020102BFBD16D
:10835000C023124A9B02116B194080235B050B431B
:108360000F498B4214D00F498B4209D00E4A9342D9
:10837000E8D0FFF7ADFFFFF767FFFFF771FFE3E717
:1083800012680223100018401A42DDD00748DBE7CC
:10839000106A8007C00FC003D6E7C0460010024035
:1083A00000000210000003100000011000127A000B
:1083B0000368020070B501205B062CD44E680B6880
:1083C00048693343CE68156833430E690C6A3343FA
:1083D0008E6903433343CE69000C3343104E23436D
:1083E00035402B43136053688D680E4E284333404D
:1083F0001843802350601B019D4204D280205368A3
:10840000400103435360802300209B019C4202D122
:108410004B6A9BB21361D36903490B40D36170BDB2
:108420004000FFFFFBF0FFFFFFF7FFFF10B5204C00
:108430000368A04206D08022D205904202D01D4A95
:1084400090420CD1702293434A681343A04212D049
:108450008022D20590420ED0164A90420BD0164A86
:10846000904208D0154A904205D0154A904202D059
:10847000144A904203D1144A1A40CB681343036054
:108480008B68C3620B888362A04208D00B4B984272
:1084900005D00B4B984202D00A4B984201D10B6990
:1084A00003630123426913434361002010BDC046AA
:1084B000002C01400004004000200040004001402A
:1084C0000044014000480140FFFCFFFF802370B5DD
:1084D0005B00994200D1A7E005D8012932D01029CC
:1084E00066D0012070BD80235B019942F9D1036AF7
:1084F0006A4E6B4C33400362056A4168C36923408E
:10850000146824021C43674B1D4013691B032B4353
:10851000556833402D032B43634DA84208D0634D6B
:10852000A84205D0624DA84202D0624DA84204D1B3
:10853000614D0D40916989012943D2684160C46150
:10854000026433E07326036A8B430362036A446860
:108550008569B543166835430226B343166933432C
:108560008B4351680B435049884208D04F49884299
:1085700005D04F49884202D04E49884212D1082185
:108580008B435169890019430423994393689B00E5
:108590000B434A49214094692143494C2140D46905
:1085A00064000C43D268446085614263036239E031
:1085B000036A3B4C8B430362066A43688569254026
:1085C000146824022C432025AE4315692D01354340
:1085D0008D43290055682D010D433349884208D049
:1085E0003249884205D03249884202D03149884216
:1085F00013D180218D435169890129434025A94325
:108600009568AD010D432F490B40916989001943CD
:108610002D4B1940D369DB000B434360D368846161
:108620008363056200205DE77321036A234E3340B4
:108630000362056A4368C4698C4311680C4320498E
:108640000D40116909022943556831402D020D433F
:108650001549884208D01549884205D014498842F6
:1086600002D01449884213D117490D40516989023B
:108670002943144D29409568AD020D4307490B402D
:10868000916909011943074B1940D3695B010B43F9
:108690004360D368C461C363C3E7C046FFEFFFFF15
:1086A000FF8CFFFFFFDFFFFF002C01400040014077
:1086B0000044014000480140FFBFFFFFFFFEFFFFF5
:1086C000FFFDFFFFFFFBFFFFFFF7FFFF1B4A03005C
:1086D00090420BD180221A4BD201D9680A43DA604A
:1086E000DA6818490A40DA6000207047164A90425A
:1086F0000AD18022124B920219690A431A611A693F
:1087000012490A401A61EFE7114A904208D18022CB
:108710000B4BD20219690A431A611A690D49F0E735
:108720000D4A01209342E0D18022054B12031969C2
:108730000A431A611A690949E3E7C0460038014053
:1087400000100240FFBFFFFF00440040FFFFFDFF9D
:1087500000480040FFFFFBFF004C0040FFFFF7FF19
:10876000026830B50123040010000D0085B01840E8
:108770001A4202D0012005B030BD4B68C96822689A
:108780000B4329690B43A9690B4321490A40134351
:10879000236063681F4A1340AA6813436360A36899
:1087A0001D4A13406A691343A3601C4B9C4218D1B5
:1087B000FFF7BAFD0028DDD029680029DAD0802231
:1087C000AD694B08120295421CD14000C018F7F762
:1087D000B7FC134B03400007400F1843E060002034
:1087E000C9E7104B9C4201D11020E1E70E4B9C429F
:1087F00004D101A8FFF78CFD0398DBE70B4B9C42EB
:10880000B8D1F6E7C018F7F79BFC80B2E6E7C046A0
:10881000F369FFEFFFCFFFFFFFFCFFFF00380140D0
:10882000F0FF00000044004000480040004C0040C1
:1088300070B53024164DA84213D80C70FA2430219C
:10884000A400A04213D211703022632815D81A70E8
:108850003023092816D8049A30301370059B1870FD
:1088600070BD0C4E01348019E4B280B2E3E70A4DCA
:1088700001314019C9B280B2E3E701326438D2B2A3
:1088800080B2E2E701330A38DBB280B2E1E7C046EA
:108890000F270000F0D8FFFF18FCFFFF13B50C00F6
:1088A0008B1C4A1C04310191E11C00912100FFF74F
:1088B000BFFF0023637113BD0209130037339F28E4
:1088C00000D8073B0B700F231840030037330928EB
:1088D00000D8073B4B7000238B70704710B5034CDA
:1088E0002100FFF7E9FF200010BDC046D816002088
:1088F00013B50B006946CB71036807319C680123EF
:10890000A04713BD13B56B460268D97107331469CC
:1089100019000122A04713BDF8B504000F001D0087
:10892000036816005B699847236820001B68984716
:1089300039002000221DFFF7DBFF002D05D0236842
:108940002A00310020001B699847236820005B68DB
:10895000984723680C2120009B699847F8BDF8B51B
:1089600004000F0015001E0003685B699847236828
:1089700020001B6898473900221D2000FFF7B8FF30
:1089800020000021FFF7BEFF2368320029002000ED
:10899000DB689847236820005B689847F8BDF8B506
:1089A00004000D0016001F0003685B6998472368E8
:1089B00020001B689847221D20001821FFF798FF10
:1089C000290A2000FFF79EFFE9B22000FFF79AFF77
:1089D00023683A00310020001B6998472368200073
:1089E0005B68984723680C2120009B699847F8BD75
:1089F00007B513006A46073213700123FFF7CFFF54
:108A000007BDF8B504000D0016001F0003685B6980
:108A10009847236820001B689847221D20001921D1
:108A2000FFF766FF290A2000FFF76CFFE9B220007C
:108A3000FFF768FF20000021FFF764FF23683A007A
:108A400031002000DB689847236820005B68984766
:108A5000F8BD13B56B46DC1D22000123FFF7D1FFE3
:108A6000207816BDF8B504000F0015001E0003683D
:108A70005B699847236820001B689847221D2000E7
:108A80001A21FFF735FF39002000FFF73BFF23686D
:108A90003200290020001B699847236820005B688A
:108AA000984723680C2120009B699847F8BDF8B5CA
:108AB00004000F0015001E0003685B6998472368D7
:108AC00020001B689847221D20001B21FFF710FF84
:108AD00039002000FFF716FF20000021FFF712FFEA
:108AE0002368320029002000DB68984723682000B3
:108AF0005B689847F8BD000037B56B460400DA1D87
:108B0000117001230D008021FFF706FF2368322139
:108B10009B69012D00D002492000984737BDC0460F
:108B2000DC05000007B56B46DA1D117001238A21B0
:108B3000FFF7F2FE07BD07B50B0C01AA13700B0A75
:108B40005370917003238621FFF7E6FE07BD07B53A
:108B50006B4619715A718F21022301AAFFF7DCFEBF
:108B600007BD000037B50C0001A94A708B700A00E0
:108B70000C7003238B210500FFF7CEFE702C13D061
:108B80000ED8EF23503C1C420CD11E22280007496E
:108B9000FFF72EFF280001220549FFF729FF37BD07
:108BA000802C01D03222F1E73722EFE725090000BF
:108BB0003C09000073B56E46B370002306AC2578FF
:108BC00007AC2478317072707371B3716A468C216E
:108BD0000733F5703471FFF79FFE73BD37B56D46EF
:108BE00006AC248849BA52BA5BBA29806A80AB8045
:108BF0006A4608238D2164BAEC80FFF78DFE37BDED
:108C000007B5022301AA1521FFF7A9FE6B466A46A4
:108C10001B7950791B02C01880B20EBD07B549BA46
:108C200001AA118002239721FFF776FE07BD70B5D8
:108C30000E000400FFF7E4FF050031002000FFF7FD
:108C4000EDFF280070BD07B50B1C1F2900D91F239D
:108C500069460B714A7102238E2101AAFFF75CFE5F
:108C600007BD130013B5040001AA1170190A517051
:108C7000937083210323FFF74FFE236864212000B4
:108C80009B69984713BD130013B5040001AA117026
:108C9000190A5170937082210323FFF73DFE236868
:108CA000642120009B69984713BD37B505230C004C
:108CB00015001D216A46FFF752FE6B461B78F02B0C
:108CC00002D900236A4613706B461B7801225B08A9
:108CD0005B4223806B4603219A56D3170B409B18A7
:108CE0009B102B70033202DA2288D318238037BD01
:108CF00037B502230D001400172101AAFFF72FFE3C
:108D00006B461B792B706B465B79237037BD07B5BB
:108D10006B46DA1D117001239E21FFF7FDFD07BD93
:108D2000002310B504001A00C121FFF7F5FD2368E8
:108D3000462120009B69984710BD000070B50D00CA
:108D400009490400FFF785FE0200012D08D14023E8
:108D50005B421A43D2B220000349FFF749FE70BDBF
:108D60003F231A40F7E7C04691080000542170B530
:108D7000FF310500FFF76DFEAA210400490028001D
:108D8000FFF767FE2402204380B270BD13B501AC2B
:108D900021706270A370220003238B21FFF7BCFDBA
:108DA00013BD0000F7B59C466B465A70624604003E
:108DB00008A8077809A806780AA80078DF701E714D
:108DC00019709A7058716A460823200093718C219B
:108DD0000BAD013B2D88FFF79FFD6B466DBA1D80E3
:108DE0006A46022320000249FFF7D9FDF7BDC046BD
:108DF000C809000073B514000D0C0B0A0E0E09BA59
:108E0000022201912100EDB29143DBB201AA0029B7
:108E10001DD101248C2E04D1382D02D10E4C14808A
:108E20000C00117863290CD151780E2909D10B4916
:108E30000024118008218B43190080235B420B43DF
:108E4000937004230649FFF7AAFD200076BD043C79
:108E5000631E9C41E4B2F4E7ACA9FFFF6B2A00005B
:108E6000CF09000013B505230C006A461D21FFF74A
:108E700076FD6B461B785B085B42238013BD0000C8
:108E8000C30DDBB27F3B020010B5162B13DC002BA9
:108E900007DAC20FD007013302D1FE239B05184326
:108EA00010BD084919410142FAD08020C003184181
:108EB00080188843F4E7802BF2D1011CF7F742FBBE
:108EC000EEE7C046FFFF7F0010B5884202D98B183D
:108ED000984203D3002307E08B5C8354013AFBD212
:108EE00010BDCC5CC45401339A42FAD1F8E70300B8
:108EF0008218934200D1704719700133F9E70200DC
:108F000010B5137814000132002BFAD1CA5CE25478
:108F10000133002AFAD110BDC9B20378002B04D066
:108F20008B4200D170470130F7E74B42594149422B
:108F30000840F7E730B50500101E0BD00024013AB9
:108F40002B5D085D834204D1A24202D00134002B84
:108F5000F6D1181A30BD000070B500260C4C0D4D2E
:108F6000641BA410A64209D1002600F02BF80A4C7D
:108F70000A4D641BA410A64205D170BDB300EB5886
:108F800098470136EEE7B300EB5898470136F2E711
:108F90008CA900088CA9000894A900088CA90008D5
:108FA00003000A7801311A700133002AF9D17047A1
:108FB000002310B59A4200D110BDCC5CC4540133DB
:108FC000F8E70000F8B5C046F8BC08BC9E467047FC
:0C8FD000F8B5C046F8BC08BC9E467047CF
:108FDC005C0A0008EA0900083E090008F6080008C7
:108FEC003E090008260A00083E090008F608000899
:108FFC00EA090008EA090008260A0008F608000831
:10900C00FC080008FC080008FC080008340A0008EA
:10901C00EA090008EA0900083E090008F2080008FD
:10902C003E090008260A00083E090008F20800085C
:10903C00EA090008EA090008260A0008F2080008F4
:10904C00FC080008FC080008FC080008300A0008AE
:10905C006D696E2C00206D572C0020572C00322E81
:10906C003447003931354D003836384D0034333300
:10907C004D003730636D003836364D003F003530CB
:10908C00487A003331487A003139487A00464C52DC
:10909C00430046534B003139487A377800011F138F
:1090AC006F01130000D57FAAFE2B815429FC568337
:1090BC00D702A87D52872DF8AC79D3067BAE04D1AC
:1090CC008550FA2FA471DB0E5A8F25F08D58F2279C
:1090DC0073A60CD9F623895C08DD77A2DF0AA0758C
:1090EC0021F45E8B9D48E23763B61CC9B461CB1E7C
:1090FC004A9F35E0CF1AB06531E44E9BE633994C6C
:10910C0018CD67B239EC4693C712B86D10C56FBA5B
:10911C00EE3B91446BBE14C19540EA3F42973DE84B
:10912C00BC69C316EF3A904511C46EBBC613B96C3B
:10913C0038ED4792BD68C21743963CE99441EB3E2B
:10914C006ABF15C04B9E34E1B560CA1F62B71DC81B
:10915C009C49E33619CC66B3E732984D30E54F9A0B
:10916C00CE1BB16472A70DD88C59F3265B8E24F1FB
:10917C00A570DA0F20F55F8ADE0BA17409DC76A3EB
:10918C00F722885DD603A97C28FD5782FF2A8055DB
:10919C0001D47EAB8451FB2E7AAF05D0AD78D207CB
:1091AC0053862CF96162636465666768696A6B6CE7
:1091BC006D6E6F707172737475767778797A3031F1
:1091CC0032333435363738395F232D2E000000000A
:1091DC000000000000000000851D000800000000D9
:1091EC0000000000911D00080000000000000000BD
:1091FC00691D00086D6C72732E30005365747570A8
:10920C005374617274537478345278005365747566
:10921C007053746172744D61726B65720021656E6E
:10922C00642100466C79536B792046524D333033B0
:10923C00006D4C525301020304006D4C5253040355
:10924C000201000A0040504152414D2F7061726181
:10925C006D2E70636B006661696C20610020005399
:10926C0078206E6F74206F6B002E000000000000E1
:10927C0000000000CD1F0008D91F00085529000868
:10928C0089290008AF29000859250008551F000836
:10929C00793B00080000000000000000AF1E000831
:1092AC00612D00082D2C0008B51E0008672B000846
:1092BC00E51F0008D12B0008F51F0008992B0008AA
:1092CC00192000080000000000000000AF1E00087C
:1092DC00B11E0008B31E0008B51E0008B91E000818
:1092EC00BB1E0008BF1E0008C31E0008C51E0008D8
:1092FC00C91E00080000000000000000E34A00083E
:10930C00814B0008654B0008454B0008000000002D
:10931C0000000000AF1E00081D200008B31E00084E
:10932C00B51E0008315300081F20000881530008A7
:10933C0031210008C51E0008C91E000800010205E5
:10934C000304800CD007B704C71B800CB7040410AF
:10935C00020A0B06972304100B060000B4A50008A4
:10936C005000000038A900080300000000000000B5
:10937C0000000000000000000000000000000000E1
:10938C0000000000000000000000000000000000D1
:10939C0000000000000000000000000000000000C1
:1093AC0000000000000000000000000000000000B1
:1093BC00000000000000000000000000800080FFA2
:1093CC00140064001800FA001B00F4011E00E803EE
:1093DC006162636465666768696A6B6C6D6E6F70F9
:1093EC007172737475767778797A303132333435AB
:1093FC00363738395F232D2E0000000000000000A6
:10940C003209000000000000010000007C2B00006D
:10941C000000000002000000890C000000000000A9
:10942C0004000000ED0E030C0D0000000500000010
:10943C00D91C0100000000000600000068030000B9
:10944C000000000007000000772000000000000072
:10945C000800000075240000000000000B00000054
:10946C0059060104000000001300000089180304D1
:10947C000500000014000000D614030203000000D5
:10948C00150000009F020300010000001600000000
:10949C00DC1900000000000017000000A8170304EE
:1094AC000500000018000000183400000000000047
:1094BC001900000017650000000000001A000000F1
:1094CC00AA180000000000001B000000901D000006
:1094DC00000000001C000000431000000000000011
:1094EC001D00000073100000000000001E000000B2
:1094FC00271C0000000000001F000000F6300000D8
:10950C000000000020000000B91C0000000000005A
:10951C0021000000681C0000000000002200000078
:10952C00ED1600000000000023000000F4160000FF
:10953C000000000024000000DE25000000000000F8
:10954C0025000000D40703040500000026000000DD
:10955C00090703040500000027000000FE26032075
:10956C002100000028000000E605030203000000B3
:10957C00290000001C040302030000002A00000064
:10958C001C120000000000002B00000084030300EC
:10959C00010000002C000000DD09030203000000A4
:1095AC002D000000E8030300010000002E00000065
:1095BC000B020000000000002F00000099080300BF
:1095CC0001000000300000002915010C0000000013
:1095DC0031000000271400000000000032000000E1
:1095EC004E2503121300000033000000C4050302D3
:1095FC00030000003500000003050000000000001F
:10960C00360000000F1B0318190000003700000083
:10961C0003190000000000003D000000A7480000F6
:10962C00000000003E000000B71A0000000000001F
:10963C003F00000077B50000000000004000000073
:10964C00BFE100000000000041000000762A00008D
:10965C00000000004200000094060302030000001A
:10966C00430000001504000000000000450000004D
:10967C00F31E010A00000000460000007C260310C7
:10968C0011000000490000002626032021000000E4
:10969C004A00000014140000000000004B00000001
:1096AC009E23031E1F0000004C0000009821031E87
:1096BC001F0000004D0000008F0A03080900000085
:1096CC00500000000E0403020300000051000000D3
:1096DC006A16000000000000520000003133032421
:1096EC0025000000530000001625000000000000BB
:1096FC00540000008F350332330000005500000089
:10970C008C330000000000005600000005350332C9
:10971C0033000000570000009633000000000000EA
:10972C0059000000E71C0000000000005A00000077
:10973C00B7380000000000005B0000003F2A00006A
:10974C00000000005C00000036210000000000005A
:10975C005D0000002F5100000000000064000000BC
:10976C00AF220000000000006500000066750000DC
:10977C0000000000660000009E7500000000000064
:10978C0067000000D03900000000000068000000F5
:10979C003874000000000000690000005D3F00000C
:1097AC00000000006A0000008A2C0000000000008D
:1097BC006B0000006C410000000000006C00000019
:1097CC00205C0000000000006D000000B9090000E2
:1097DC00000000006E00000054FE030102000000B7
:1097EC006F00000022120310110000007000000036
:1097FC00AE0C000000000000710000007C2700008F
:10980C000000000072000000ED2C000000000000C1
:10981C007300000004400000000000007400000011
:10982C004C180000000000007500000080060304C6
:10983C000500000076000000380E0000000000005B
:10984C0077000000740C030A0B0000007800000085
:10985C00866100000000000079000000ED020300AA
:10986C00010000007A000000CB02030001000000A0
:10987C007B000000FA710300010000007C00000076
:10988C0057390000000000007D000000CB060000EE
:10989C00000000007E000000DC51034F500000006F
:1098AC007F00000019230000000000008000000071
:1098BC00E223000000000000810000002E180000D0
:1098CC0000000000820000001D0D000000000000E0
:1098DC0083000000DFFF0000000000008400000097
:1098EC005527000000000000850000000612000053
:1098FC000000000086000000E52B000000000000C6
:10990C0087000000CB080000000000008800000069
:10991C00011600000000000089000000C3100000C8
:10992C00000000008A0000006D78000000000000BC
:10993C008B000000A82B03292A0000008C000000DB
:10994C00B5290000000000008D0000002F20000051
:10995C00000000008E00000048F300000000000032
:10996C008F00000083100000000000009000000039
:10997C007F5D0000000000009200000067640000A2
:10998C0000000000930000009A3600000000000068
:10999C0094000000B24E0000000000009500000092
:1099AC00C83C00000000000096000000862A000061
:1099BC000000000097000000DB0803060700000011
:1099CC0098000000D0080000000000009900000082
:1099DC00BC0C0000000000009A000000540F0306AD
:1099EC00070000009B000000160D0304050000009A
:1099FC009C00000013060300010000009D00000005
:109A0C00150F030C0D0000009E000000860F030CC8
:109A1C000D000000A00000004E0C0308090000001F
:109A2C00A10000004403030001000000A20000009C
:109A3C00BD09000000000000A30000007F1C000016
:109A4C0000000000A40000009A2C000000000000A0
:109A5C00A50000001503000000000000A600000097
:109A6C001509000000000000A7000000901600007F
:109A7C0000000000A8000000010C00000000000025
:109A8C00A9000000EA12000000000000AA0000007B
:109A9C004922000000000000AB000000B5420000AD
:109AAC0000000000AC000000166200000000000086
:109ABC00AD0000005308000000000000AE000000E4
:109ACC00A730000000000000AF0000008A13030E56
:109ADC000F000000B0000000EA03030001000000CA
:109AEC00B1000000F014000000000000B200000003
:109AFC002F18000000000000B3000000BD1D011A6B
:109B0C0000000000B4000000342F012A0000000007
:109B1C00B5000000AE04000000000000B60000001C
:109B2C00E528000000000000B7000000550203000B
:109B3C0001000000B80000009FCE030405000000E7
:109B4C00B9000000BA07030405000000BA000000C9
:109B5C00481D030001000000BF0000005C1B00005A
:109B6C0000000000C00000002436000000000000CF
:109B7C00C1000000471A000000000000C2000000F5
:109B8C006221000000000000C300000078250000E6
:109B9C0000000000C8000000862A032829000000ED
:109BAC00C9000000CD0E030C0D000000D600000013
:109BBC004508030607000000D700000065030000FD
:109BCC0000000000D8000000320303000100000078
:109BDC00D9000000CA06000000000000DA000000F6
:109BEC001107030001000000DB000000A2020000CE
:109BFC0000000000DC00000022200000000000003B
:109C0C00DD000000472A000000000000DE0000001C
:109C1C000F03000000000000DF000000772F032A74
:109C2C002B000000E0000000662D032A2B00000032
:109C3C00E1000000D049000000000000E20000003C
:109C4C00CF08000000000000E6000000A32A00007E
:109C5C0000000000E7000000692800000000000080
:109C6C00E80000009741000000000000E90000003F
:109C7C0023B6000000000000EA0000009628000057
:109C8C0000000000EB000000B32A00000000000000
:109C9C00F10000005A20000000000000F20000005B
:109CAC00683C000000000000F3000000553D01344A
:109CBC0000000000F40000005F060000000000003F
:109CCC00F50000008202000000000000F600000019
:109CDC00B826000000000000F7000000511300003F
:109CEC0000000000F800000008FE03030400000060
:109CFC00F9000000CC24000000000000FA00000075
:109D0C00311E000000000000FB000000AA12000041
:109D1C0000000000FC0000002C12000000000000FD
:109D2C00FD0000005336000000000000FE000000A3
:109D3C002E0900000000000000010000472A030863
:109D4C000900000001010000830900000000000070
:109D5C0002010000BBE80300010000000301000049
:109D6C005CED00000000000004010000920E0000F9
:109D7C000000000005010000B33D000000000000E1
:109D8C00060100000C170000000000000701000095
:109D9C0085FF0000000000000801000031200000D9
:109DAC0000000000090100001A140000000000006F
:109DBC000A010000C1FF0302030000000B010000B8
:109DCC0023FF0302030000000C0100000E04030239
:109DDC00030000000D0100006DD700000000000022
:109DEC000E0100003B140000000000000F010000F9
:109DFC001635000000000000130100007E2000005A
:109E0C0000000000140100001232000000000000ED
:109E1C00150100003E1E00000000000018010000AB
:109E2C00462100000000000019010000300D000068
:109E3C00000000001A0100007B2303202100000019
:109E4C001B0100004A910000000000001C010000F2
:109E5C006320031E1F0000001D0100008931032632
:109E6C00270000001E010000D2390332330000002D
:109E7C001F01000001170314150000002001000051
:109E8C00141703141500000022010000FB2E000023
:109E9C0000000000230100000A390000000000004F
:109EAC0027010000EA0C0000000000002A0100005D
:109EBC00ED250000000000002B01000013620000E3
:109ECC00000000002C010000D9160000000000006A
:109EDC002D010000F33A00000000000036010000E4
:109EEC001C11000000000000370100005F7400002E
:109EFC000000000040010000F31403020300000006
:109F0C004101000058020300010000004201000062
:109F1C00F395000000000000430100004E93030085
:109F2C0001000000440100008492000000000000C9
:109F3C004A01000017A70000000000004B010000C0
:109F4C005BE90000000000004C010000ECEF000099
:109F5C00000000004D010000E76D00000000000053
:109F6C004E010000480A0000000000004F010000F4
:109F7C00E11800000000000050010000F554000042
:109F8C000000000053010000C705000000000000A5
:109F9C005401000063460000000000005E01000058
:109FAC00E8FC00000000000062010000D20E030C6F
:109FBC000D00000063010000060C00000000000012
:109FCC00680100000B19000000000000690100008E
:109FDC005D210000000000007101000097180000D6
:109FEC0000000000720100001A8C0000000000004C
:109FFC00730100000A1A0000000000007501000047
:10A00C00752A00000000000077010000FB8C0000A6
:10A01C000000000078010000C708000000000000EC
:10A02C007C010000E8140000000000008101000029
:10A03C0093850302030000008201000084100304D6
:10A04C000500000083010000044803040500000023
:10A05C008401000008250320210000008601000077
:10A06C009CEE0000000000008B01000000D40000FA
:10A07C00000000008C01000032A000000000000075
:10A08C008D010000B66C0000000000009001000083
:10A09C006EFE03040500000091010000B7060304E6
:10A0AC00050000009A010000A0350000000000002F
:10A0BC009B0100006A030000000000009C010000EE
:10A0CC0021060304050000009D0100004D07030458
:10A0DC00050000009E0100006D1000000000000053
:10A0EC009F010000A110000000000000A40100006E
:10A0FC001449030607000000B3010000862E00007F
:10A10C0000000000B4010000C109000000000000C4
:10A11C00B50100001E01000000000000B8010000A5
:10A12C004223000000000000B9010000A91100004A
:10A13C0000000000FE010000F56A000000000000B5
:10A14C00FF0100001C47000000000000421F00003F
:10A15C00DA10000000000000431F0000E729000097
:10A16C0000000000441F0000AC6200000000000072
:10A17C00451F0000FB26000000000000461F0000E9
:10A18C00610E000000000000471F0000402000008E
:10A19C0000000000481F0000EA2100000000000041
:10A1AC00491F000090100000000000004A1F000032
:10A1BC009B290000000000004B1F000014660000EB
:10A1CC00000000004C1F00003610000000000000D2
:10A1DC004D1F0000DE2E0000000000004E1F00008E
:10A1EC00C80E0000000000004F1F000017180000F0
:10A1FC0000000000501F000095120000000000003D
:10A20C002823000071890000000000002D230000AD
:10A21C00752200000000000011270000D11400007E
:10A22C000000000012270000BA2900000000000006
:10A23C00132700000401000000000000A727000005
:10A24C00C355000000000000F82A00008634030407
:10A25C0005000000F92A00000F8800000000000033
:10A26C00FA2A0000EAB4030405000000FB2A0000EF
:10A27C004005000000000000FC2A00000BE8030869
:10A28C0009000000FD2A00005DE60000000000004F
:10A29C00022B00002E31000000000000032B0000F8
:10A2AC006A2C0000000000000C2B0000CD100000F8
:10A2BC0000000000162B0000902C00000000000095
:10A2CC00172B0000852C000000000000182B00004C
:10A2DC00552C000000000000192B0000C3250310B2
:10A2EC00110000001A2B00004F05000000000000B8
:10A2FC001B2B000080080304050000001C2B000031
:10A30C00B1220000000000001D2B0000821C000088
:10A31C00000000001E2B00002F2600000000000093
:10A32C001F2B00008E09000000000000202B0000F5
:10A33C00842C000000000000212B0000D02C000019
:10A34C0000000000222B0000C92C000000000000BF
:10A35C00232B0000C12C000000000000242B000067
:10A36C00BD2C00000000000064320000722C0300C1
:10A37C000100000065320000FE3B031E1F000000C0
:10A38C00663200008C3503040500000067320000C3
:10A39C00F92E030001000000683200004D36031C4A
:10A3AC001D00000069320000312B03000100000089
:10A3BC00733200005EF903000100000076320000E9
:10A3CC008B330000000000007732000007120310EE
:10A3DC00110000007832000014050000000000009D
:10A3EC006842000067B3000000000000FE4200005D
:10A3FC001A21000000000000FF420000481000007D
:10A40C0000000000014300001311000000000000D8
:10A41C00024300005911000000000000034300003B
:10A42C001B0A000000000000044300000E5B00004B
:10A43C000000000005430000BB54000000000000B9
:10A44C00064300006A1800000000000010A4000081
:10A45C00E30100000000000011A40000EF2E00003A
:10A46C000000000051C30000F620000000000000B6
:10A47C0052C30000B5F600000000000053C30000FA
:10A48C003E1300000000000054C30000F00A030853
:10A49C000900000055C300009806030405000000E5
:10A4AC0020CB00000D6400000000000021CB000058
:10A4BC00EF0100000000000022CB0000180100009A
:10A4CC000000000023CB0000A61A000000000000D2
:10A4DC0024CB0000270100000000000025CB000069
:10A4EC00910100000000000060EA00000416031453
:10A4FC00150000006AEA0000D021000000000000F6
:10A50C006BEA0000B7070000000000006CEA0000D6
:10A51C0063240320210000006DEA0000811803145D
:10A52C00150000006EEA0000860803040500000018
:10A53C0074EA0000CA0400000000000088EA000071
:10A54C009CF500000000000089EA0000BFFF00003D
:10A55C00000000008DEA00000E170302030000004B
:10A56C008EEA0000AB1C0308090000008FEA000013
:10A57C00370700000000000092EA0000DC0E00002B
:10A58C000000000093EA0000F51800000000000035
:10A59C0094EA0000652C00000000000095EA000021
:10A5AC002D060000000000003BB1B800ECC4B80060
:10A5BC009DD8B8004EECB8000000B900B113B9003A
:10A5CC006227B900133BB900C44EB9007662B900DA
:10A5DC002776B900D889B900899DB9003BB1B9007B
:10A5EC00ECC4B9009DD8B9004EECB9000000BA001B
:10A5FC00B113BA006227BA00133BBA00C44EBA00BA
:10A60C007662BA002776BA00D889BA00899DBA005A
:10A61C003BB1BA00ECC4BA009DD8BA004EECBA00FB
:10A62C000000BB00B113BB006227BB00133BBB0097
:10A63C00C44EBB007662BB002776BB00D889BB003A
:10A64C00899DBB003BB1BB00ECC4BB009DD8BB00DB
:10A65C004EECBB000000BC00B113BC006227BC0078
:10A66C00133BBC00C44EBC007662BC002776BC0019
:10A67C00D889BC00899DBC003BB1BC00ECC4BC00BB
:10A68C009DD8BC004EECBC000000BD00B113BD0059
:10A69C006227BD00133BBD00C44EBD007662BD00F9
:10A6AC002776BD00D889BD00899DBD003BB1BD009A
:10A6BC00ECC4BD009DD8BD004EECBD000000BE003A
:10A6CC00B113BE006227BE00133BBE00C44EBE00D9
:10A6DC007662BE002776BE00D889BE00899DBE007A
:10A6EC003BB1BE00ECC4BE000000891112239B32AA
:10A6FC002446AD573665BF74488CC19D5AAFD3BE46
:10A70C006CCAE5DB7EE9F7F88110080193331A2255
:10A71C00A5562C47B7753E64C99C408DDBBF52AE25
:10A72C00EDDA64CBFFF976E802218B301002991335
:10A73C002667AF763444BD554AADC3BC588ED19F05
:10A74C006EEBE7FA7CC8F5D983310A209112180315
:10A75C00A7772E66B5543C45CBBD42ACD99E508FE5
:10A76C00EFFB66EAFDD874C904428D5316619F70E5
:10A77C002004A9153227BB364CCEC5DF5EEDD7FCC5
:10A78C006888E1997AABF3BA85520C4397711E60D5
:10A79C00A1142805B3373A26CDDE44CFDFFD56ECA5
:10A7AC00E9986089FBBB72AA06638F7214409D51B5
:10A7BC002225AB343006B9174EEFC7FE5CCCD5DD85
:10A7CC006AA9E3B8788AF19B87730E6295501C4195
:10A7DC00A3352A24B1163807CFFF46EEDDDC54CD65
:10A7EC00EBB962A8F99A708B088481951AA793B675
:10A7FC002CC2A5D33EE1B7F04008C919522BDB3A65
:10A80C00644EED5F766DFF7C899400859BB712A634
:10A81C00ADD224C3BFF136E0C1184809D33B5A2A44
:10A82C00E55E6C4FF77D7E6C0AA583B41886919714
:10A83C002EE3A7F23CC0B5D14229CB38500AD91B24
:10A84C00666FEF7E744CFD5D8BB502A499961087F4
:10A85C00AFF326E2BDD034C1C3394A28D11A580B04
:10A86C00E77F6E6EF55C7C4D0CC685D71EE597F4C4
:10A87C002880A1913AA3B3B2444ACD5B5669DF78E4
:10A88C00600CE91D722FFB3E8DD604C79FF516E4B4
:10A89C00A9902081BBB332A2C55A4C4BD7795E68C4
:10A8AC00E11C680DF33F7A2E0EE787F61CC495D594
:10A8BC002AA1A3B03882B193466BCF7A5448DD59A4
:10A8CC00622DEB3C700EF91F8FF706E69DD414C574
:10A8DC00ABB122A0B9923083C77B4E6AD5585C4984
:10A8EC00E33D6A2CF11E780F860010700410005B9B
:10A8FC000000E86A4F09000098FF00005018050C92
:10A90C00805B0040D41E000097FF00006018050C0F
:10A91C00805B00406A34000094FF00007018050C46
:10A92C00805B0040E75B000090FF00002E0E4400AF
:10A93C000000000000000000816D0008836D00081D
:10A94C00876D00088B6D00080000000000000000FF
:10A95C0001020304060708090000000001020304B9
:10A96C0002030405060708090A0B0C0D0E0F101044
:10A97C000102030405060708090A0B0C0D0E0F1043
:08A98C00E9000008316D00082C
:04A99400C1000008F6
:10A9980090BADCFE785634120A000000D8920008FB
:10A9A800A8920008FF0000002093000800127A0017
:08A9B800010000000400000092
:040000050800764930
:00000001FF
